 ARTLOOK

 Timestamp is 417c0e2b (Sun Oct 24 13:18:51 2004)

 Preferred load address is 00010000

 Start         Length     Name                   Class
 0001:00000000 000331e1H .text                   CODE
 0002:00000000 0000a0e9H .bss                    DATA
 0003:00000000 00000300H .rdata                  DATA
 0004:00000000 00009204H .data                   DATA
 0004:00009208 00000004H .CRT$XCA                DATA
 0004:00009210 00000004H .CRT$XCZ                DATA
 0004:00009218 00000004H .CRT$XIA                DATA
 0004:0000921c 00000008H .CRT$XIC                DATA
 0004:00009228 00000004H .CRT$XIF                DATA
 0004:00009230 00000004H .CRT$XIG                DATA
 0004:00009240 00000004H .CRT$XIX                DATA
 0004:00009248 00000004H .CRT$XIZ                DATA
 0004:00009250 00000004H .CRT$XPA                DATA
 0004:00009254 00000008H .CRT$XPX                DATA
 0004:00009260 00000004H .CRT$XPZ                DATA
 0004:00009268 00000004H .CRT$XTA                DATA
 0004:00009270 00000004H .CRT$XTZ                DATA
 0005:00000000 00000009H _CONST                  DATA
 0006:00000000 00000014H .idata$2                DATA
 0006:00000014 00000014H .idata$3                DATA
 0006:00000028 00000100H .idata$4                DATA
 0006:00000128 00000100H .idata$5                DATA
 0006:00000228 0000047eH .idata$6                DATA
 0008:00000000 000333cdH .debug$C                DATA
 0008:000333d0 00001760H .debug$F                DATA
 0008:00034b30 00000000H .debug$G                DATA
 0008:00034b30 00000008H .debug$H                DATA
 0008:00034b38 00009b50H .debug$S                DATA
 0008:0003e688 00007597H .debug$T                DATA

  Address         Publics by Value              Rva+Base   Lib:Object

 0001:fffff000       ___getviewcoord_w          00010000   libf:qcdumb.obj
 0001:fffff000       ___nmalloc                 00010000   libf:qcdumb.obj
 0001:fffff000       ___nfree                   00010000   libf:qcdumb.obj
 0001:fffff000       ___aFldiv                  00010000   libf:qcdumb.obj
 0001:fffff000       ___getcurrentposition_w    00010000   libf:qcdumb.obj
 0001:fffff000       ___acrtused                00010000   libf:qcdumb.obj
 0001:fffff000       ___getwindowcoord          00010000   libf:qcdumb.obj
 0001:fffff000       ___getviewcoord_wxy        00010000   libf:qcdumb.obj
 0001:fffff000       ___memmax                  00010000   libf:qcdumb.obj
 0001:00000000       _MOUSEINIT@0               00011000 f MOUSE.OBJ
 0001:000000e5       _GETMOUSEEVENT@4           000110e5   MOUSE.OBJ
 0001:000001cd       _GETPTRPOS@4               000111cd   MOUSE.OBJ
 0001:0000027c       _SETPTRPOS@8               0001127c   MOUSE.OBJ
 0001:000002f8       _GETBUTTONPRESS@4          000112f8   MOUSE.OBJ
 0001:000003ab       _GETBUTTONRELEASE@4        000113ab   MOUSE.OBJ
 0001:0000045e       _SETPTRVIS@4               0001145e   MOUSE.OBJ
 0001:000004a0       _main                      000114a0 f ARTLOOK.OBJ
 0001:00003e30       _DISPLB                    00014e30 f DISPLB.OBJ
 0001:00003e30       _DISPLB@68                 00014e30 f DISPLB.OBJ
 0001:000069b6       _TIMTIK@36                 000179b6 f DISPLB.OBJ
 0001:000069b6       _TIMTIK                    000179b6 f DISPLB.OBJ
 0001:00006e8f       _TIMLIN                    00017e8f f DISPLB.OBJ
 0001:00006e8f       _TIMLIN@36                 00017e8f f DISPLB.OBJ
 0001:00007220       _ARTID@16                  00018220 f INPUT.OBJ
 0001:00007220       _ARTID                     00018220 f INPUT.OBJ
 0001:000077ef       _DECOHEAD@36               000187ef f INPUT.OBJ
 0001:000077ef       _DECOHEAD                  000187ef f INPUT.OBJ
 0001:000079bd       _CNVDT@4                   000189bd f INPUT.OBJ
 0001:000079bd       _CNVDT                     000189bd f INPUT.OBJ
 0001:00007a0d       _ARTFREQ@4                 00018a0d f INPUT.OBJ
 0001:00007a0d       _ARTFREQ                   00018a0d f INPUT.OBJ
 0001:00007db9       _ARTREAD                   00018db9 f INPUT.OBJ
 0001:00007db9       _ARTREAD@28                00018db9 f INPUT.OBJ
 0001:00008584       _COPAV                     00019584 f INPUT.OBJ
 0001:00008584       _COPAV@48                  00019584 f INPUT.OBJ
 0001:00008f23       _BLOCKXTR@16               00019f23 f INPUT.OBJ
 0001:00008f23       _BLOCKXTR                  00019f23 f INPUT.OBJ
 0001:000093f0       _PREPDISP                  0001a3f0 f OUTPUT.OBJ
 0001:000093f0       _PREPDISP@52               0001a3f0 f OUTPUT.OBJ
 0001:00009c89       _SAVEART                   0001ac89 f OUTPUT.OBJ
 0001:00009c89       _SAVEART@56                0001ac89 f OUTPUT.OBJ
 0001:0000a1a3       _ARTDUMP@28                0001b1a3 f OUTPUT.OBJ
 0001:0000a1a3       _ARTDUMP                   0001b1a3 f OUTPUT.OBJ
 0001:0000a7cb       _SPECMAX                   0001b7cb f OUTPUT.OBJ
 0001:0000a7cb       _SPECMAX@28                0001b7cb f OUTPUT.OBJ
 0001:0000ac70       _CALIBR@52                 0001bc70 f PROCESS.OBJ
 0001:0000ac70       _CALIBR                    0001bc70 f PROCESS.OBJ
 0001:0000b039       _BACK                      0001c039 f PROCESS.OBJ
 0001:0000b039       _BACK@68                   0001c039 f PROCESS.OBJ
 0001:0000bacd       _BACKSUB@32                0001cacd f PROCESS.OBJ
 0001:0000bacd       _BACKSUB                   0001cacd f PROCESS.OBJ
 0001:0000bd05       _BASE                      0001cd05 f PROCESS.OBJ
 0001:0000bd05       _BASE@16                   0001cd05 f PROCESS.OBJ
 0001:0000bfdb       _BASE2@20                  0001cfdb f PROCESS.OBJ
 0001:0000bfdb       _BASE2                     0001cfdb f PROCESS.OBJ
 0001:0000c2d0       _CNGBUF@20                 0001d2d0 f CNGBUF.OBJ
 0001:0000c2d0       _CNGBUF                    0001d2d0 f CNGBUF.OBJ
 0001:0000c500       _IMSAVE@8                  0001d500 f IMSAVE.OBJ
 0001:0000c500       _IMSAVE                    0001d500 f IMSAVE.OBJ
 0001:0000cae0       _MVCURS                    0001dae0 f MVCURS.OBJ
 0001:0000cae0       _MVCURS@44                 0001dae0 f MVCURS.OBJ
 0001:0000cf40       _MOSINI                    0001df40 f FMOUSE.OBJ
 0001:0000cf40       _MOSINI@8                  0001df40 f FMOUSE.OBJ
 0001:0000cf77       _MOSGET                    0001df77 f FMOUSE.OBJ
 0001:0000cf77       _MOSGET@12                 0001df77 f FMOUSE.OBJ
 0001:0000cfb6       _MOSDIS@8                  0001dfb6 f FMOUSE.OBJ
 0001:0000cfb6       _MOSDIS                    0001dfb6 f FMOUSE.OBJ
 0001:0000d016       _CURSHO@0                  0001e016 f FMOUSE.OBJ
 0001:0000d016       _CURSHO                    0001e016 f FMOUSE.OBJ
 0001:0000d030       _KEYGET@12                 0001e030 f KEYBOARD.OBJ
 0001:0000d030       _KEYGET                    0001e030 f KEYBOARD.OBJ
 0001:0000d0f1       _KEYSTA@16                 0001e0f1 f KEYBOARD.OBJ
 0001:0000d0f1       _KEYSTA                    0001e0f1 f KEYBOARD.OBJ
 0001:0000d120       _FILEINFO@32               0001e120 f UTI.OBJ
 0001:0000d120       _FILEINFO                  0001e120 f UTI.OBJ
 0001:0000d261       _VALARGC@16                0001e261 f UTI.OBJ
 0001:0000d261       _VALARGC                   0001e261 f UTI.OBJ
 0001:0000d3b6       _VALARGR                   0001e3b6 f UTI.OBJ
 0001:0000d3b6       _VALARGR@8                 0001e3b6 f UTI.OBJ
 0001:0000d51a       _COMARG2@8                 0001e51a f UTI.OBJ
 0001:0000d51a       _COMARG2                   0001e51a f UTI.OBJ
 0001:0000d5f8       _COMARG                    0001e5f8 f UTI.OBJ
 0001:0000d5f8       _COMARG@16                 0001e5f8 f UTI.OBJ
 0001:0000d763       _CONVUC@12                 0001e763 f UTI.OBJ
 0001:0000d763       _CONVUC                    0001e763 f UTI.OBJ
 0001:0000d85c       _TIMEWR                    0001e85c f UTI.OBJ
 0001:0000d85c       _TIMEWR@16                 0001e85c f UTI.OBJ
 0001:0000d990       _TWR@12                    0001e990 f UTI.OBJ
 0001:0000d990       _TWR                       0001e990 f UTI.OBJ
 0001:0000d9e1       _TIM@4                     0001e9e1 f UTI.OBJ
 0001:0000d9e1       _TIM                       0001e9e1 f UTI.OBJ
 0001:0000da6a       _DMS@8                     0001ea6a f UTI.OBJ
 0001:0000da6a       _DMS                       0001ea6a f UTI.OBJ
 0001:0000db83       _TIMER                     0001eb83 f UTI.OBJ
 0001:0000db83       _TIMER@16                  0001eb83 f UTI.OBJ
 0001:0000dce7       _PRHEAD@20                 0001ece7 f UTI.OBJ
 0001:0000dce7       _PRHEAD                    0001ece7 f UTI.OBJ
 0001:0000decb       _XCHGI1                    0001eecb f UTI.OBJ
 0001:0000decb       _XCHGI1@8                  0001eecb f UTI.OBJ
 0001:0000defb       _XCHGI2                    0001eefb f UTI.OBJ
 0001:0000defb       _XCHGI2@8                  0001eefb f UTI.OBJ
 0001:0000df31       _XCHGI4@8                  0001ef31 f UTI.OBJ
 0001:0000df31       _XCHGI4                    0001ef31 f UTI.OBJ
 0001:0000df61       _XCHGR4@8                  0001ef61 f UTI.OBJ
 0001:0000df61       _XCHGR4                    0001ef61 f UTI.OBJ
 0001:0000df92       _XCHGR8@8                  0001ef92 f UTI.OBJ
 0001:0000df92       _XCHGR8                    0001ef92 f UTI.OBJ
 0001:0000dfdb       _XCHGS@20                  0001efdb f UTI.OBJ
 0001:0000dfdb       _XCHGS                     0001efdb f UTI.OBJ
 0001:0000e09e       _FMIN                      0001f09e f UTI.OBJ
 0001:0000e09e       _FMIN@20                   0001f09e f UTI.OBJ
 0001:0000e52e       _FMAX@20                   0001f52e f UTI.OBJ
 0001:0000e52e       _FMAX                      0001f52e f UTI.OBJ
 0001:0000e9be       _POLFIT2@28                0001f9be f UTI.OBJ
 0001:0000e9be       _POLFIT2                   0001f9be f UTI.OBJ
 0001:0000f17c       _FILTSHFT@32               0002017c f UTI.OBJ
 0001:0000f17c       _FILTSHFT                  0002017c f UTI.OBJ
 0001:00010355       _STAT2@52                  00021355 f UTI.OBJ
 0001:00010355       _STAT2                     00021355 f UTI.OBJ
 0001:00010625       _HIST2                     00021625 f UTI.OBJ
 0001:00010625       _HIST2@52                  00021625 f UTI.OBJ
 0001:00010a41       _FNAM                      00021a41 f UTI.OBJ
 0001:00010a41       _FNAM@16                   00021a41 f UTI.OBJ
 0001:00010b82       _EXTREM@16                 00021b82 f UTI.OBJ
 0001:00010b82       _EXTREM                    00021b82 f UTI.OBJ
 0001:00010cf6       _RFFT                      00021cf6 f UTI.OBJ
 0001:00010cf6       _RFFT@28                   00021cf6 f UTI.OBJ
 0001:000113b6       _FFTR@28                   000223b6 f UTI.OBJ
 0001:000113b6       _FFTR                      000223b6 f UTI.OBJ
 0001:0001174b       _DETERM                    0002274b f UTI.OBJ
 0001:0001174b       _DETERM@12                 0002274b f UTI.OBJ
 0001:00011b49       _GAUSSJ@24                 00022b49 f UTI.OBJ
 0001:00011b49       _GAUSSJ                    00022b49 f UTI.OBJ
 0001:00012530       _FFT                       00023530 f UTI.OBJ
 0001:00012530       _FFT@20                    00023530 f UTI.OBJ
 0001:00012a23       _VALARGI@8                 00023a23 f UTI.OBJ
 0001:00012a23       _VALARGI                   00023a23 f UTI.OBJ
 0001:00012b90       _DELAY                     00023b90 f DELAY.OBJ
 0001:00012b90       _DELAY@4                   00023b90 f DELAY.OBJ
 0001:00012cd0       _COLREG                    00023cd0 f COLREG.OBJ
 0001:00012cd0       _COLREG@4                  00023cd0 f COLREG.OBJ
 0001:00012f40       _CPRINT@24                 00023f40 f CPRINT.OBJ
 0001:00012f40       _CPRINT                    00023f40 f CPRINT.OBJ
 0001:00013200       _CPRINTC                   00024200 f CPRINTC.OBJ
 0001:00013200       _CPRINTC@24                00024200 f CPRINTC.OBJ
 0001:00013450       _CPRINTS                   00024450 f CPRINTS.OBJ
 0001:00013450       _CPRINTS@24                00024450 f CPRINTS.OBJ
 0001:000136a0       _GETMOD@12                 000246a0 f GETMOD.OBJ
 0001:000136a0       _GETMOD                    000246a0 f GETMOD.OBJ
 0001:000136f0       _GPRINT@28                 000246f0 f GPRINT.OBJ
 0001:000136f0       _GPRINT                    000246f0 f GPRINT.OBJ
 0001:00013b40       _HSCRLX                    00024b40 f HSCRLX.OBJ
 0001:00013b40       _HSCRLX@24                 00024b40 f HSCRLX.OBJ
 0001:00013d40       _IMCOLX                    00024d40 f IMCOLX.OBJ
 0001:00013d40       _IMCOLX@16                 00024d40 f IMCOLX.OBJ
 0001:00013e20       _IMROWX                    00024e20 f IMROWX.OBJ
 0001:00013e20       _IMROWX@16                 00024e20 f IMROWX.OBJ
 0001:00013f00       _NEGIMX@20                 00024f00 f NEGIM.OBJ
 0001:00013f00       _NEGIMX                    00024f00 f NEGIM.OBJ
 0001:000141f0       _RDCOLX@16                 000251f0 f RDCOLX.OBJ
 0001:000141f0       _RDCOLX                    000251f0 f RDCOLX.OBJ
 0001:000142d0       _RDROWX@16                 000252d0 f RDROWX.OBJ
 0001:000142d0       _RDROWX                    000252d0 f RDROWX.OBJ
 0001:000143b0       _SCREEN@0                  000253b0 f SCREEN.OBJ
 0001:000143b0       _SCREEN                    000253b0 f SCREEN.OBJ
 0001:00014650       _SETCOL                    00025650 f SETCOL.OBJ
 0001:00014650       _SETCOL@12                 00025650 f SETCOL.OBJ
 0001:0001475d       _RGB                       0002575d f SETCOL.OBJ
 0001:0001475d       _RGB@12                    0002575d f SETCOL.OBJ
 0001:000147a0       _SETMOD                    000257a0 f SETMOD.OBJ
 0001:000147a0       _SETMOD@4                  000257a0 f SETMOD.OBJ
 0001:000147e0       _SPRINT                    000257e0 f SPRINT.OBJ
 0001:000147e0       _SPRINT@28                 000257e0 f SPRINT.OBJ
 0001:00014860       _USCRLX@24                 00025860 f USCRLX.OBJ
 0001:00014860       _USCRLX                    00025860 f USCRLX.OBJ
 0001:00014a30       __getvideoconfig           00025a30   libf:qcconfig.obj
 0001:00014ad0       __FIstrcpy@24              00025ad0 f libf:intrnchr.obj
 0001:00014b70       __FIstraddr@16             00025b70 f libf:intrnchr.obj
 0001:00014b90       __FIstrcat                 00025b90 f libf:intrnchr.obj
 0001:00014c30       __FIpstrcat                00025c30 f libf:intrnchr.obj
 0001:00014d40       __FIdbgstrcpy@32           00025d40 f libf:intrnchr.obj
 0001:00014da0       __FIdbgstraddr@20          00025da0 f libf:intrnchr.obj
 0001:00014de0       __FIdbgstrcat              00025de0 f libf:intrnchr.obj
 0001:00014f70       __FIdbgpstrcat             00025f70 f libf:intrnchr.obj
 0001:000150c0       __FIvaxstrcpy@24           000260c0 f libf:intrnchr.obj
 0001:00015130       __FIvaxstrcat              00026130 f libf:intrnchr.obj
 0001:00015230       __FIpcleanup@4             00026230 f libf:intrnchr.obj
 0001:00015240       __FIclge@16                00026240 f libf:intrnchr.obj
 0001:00015270       __FIcleq@16                00026270 f libf:intrnchr.obj
 0001:000152a0       __FIclne@16                000262a0 f libf:intrnchr.obj
 0001:000152d0       __FIclgt@16                000262d0 f libf:intrnchr.obj
 0001:00015300       __FIclle@16                00026300 f libf:intrnchr.obj
 0001:00015330       __FIcllt@16                00026330 f libf:intrnchr.obj
 0001:00015360       _ccmp@16                   00026360 f libf:intrnchr.obj
 0001:00015400       __FIindex@20               00026400 f libf:intrnchr.obj
 0001:00015550       __FIlentrim@8              00026550 f libf:intrnchr.obj
 0001:00015570       __FIscan@20                00026570 f libf:intrnchr.obj
 0001:00015670       __FIverify@20              00026670 f libf:intrnchr.obj
 0001:00015770       ___FF_encflt@8             00026770 f libf:encflt.obj
 0001:00015aa0       __FFopn                    00026aa0 f libf:opn.obj
 0001:00015e70       __FFalloc                  00026e70 f libf:alla.obj
 0001:00015f40       __FFdeall                  00026f40 f libf:alla.obj
 0001:00015fd0       ___FF_inqputstr@8          00026fd0 f libf:inq.obj
 0001:00016050       __FFinq                    00027050 f libf:inq.obj
 0001:00016550       ___FF_decflt@8             00027550 f libf:decflt.obj
 0001:00016640       ___FF_nrectmo@0            00027640 f libf:nrectmo.obj
 0001:000166b0       __FFcls                    000276b0 f libf:cls.obj
 0001:000167d0       ___FF_nrectmi@0            000277d0 f libf:nrectmi.obj
 0001:00016850       ___FF_nrecfso@0            00027850 f libf:nrecfso.obj
 0001:000168a0       ___FF_nrecino@0            000278a0 f libf:nrecino.obj
 0001:00016900       __FFsSTOP                  00027900 f libf:sstop.obj
 0001:00016950       ___FF_ldout@4              00027950 f libf:ldout.obj
 0001:00016a00       ___FF_ldin@4               00027a00 f libf:ldin.obj
 0001:00016ae0       ___FF_nrecfsi@0            00027ae0 f libf:nrecfsi.obj
 0001:00016b40       ___FF_fmtout@4             00027b40 f libf:fmtout.obj
 0001:00016e20       ___FF_getchn@0             00027e20 f libf:fmtin.obj
 0001:00016f30       ___FF_fmtin@4              00027f30 f libf:fmtin.obj
 0001:000171d0       ___FF_enclong@12           000281d0 f libf:wr.obj
 0001:000172a0       __FFwr                     000282a0 f libf:wr.obj
 0001:00017380       _RUNQQ@16                  00028380 f libf:spawn.obj
 0001:00017530       _SYSTEMQQ@8                00028530 f libf:spawn.obj
 0001:00017590       ___FF_declong@4            00028590 f libf:rd.obj
 0001:00017630       ___FF_login@0              00028630 f libf:rd.obj
 0001:00017690       __FFrd                     00028690 f libf:rd.obj
 0001:00017740       ___FFmathstub              00028740   libf:intrin.obj
 0001:00017741       __FIfexp                   00028741   libf:intrin.obj
 0001:0001775b       __FIcos                    0002875b   libf:intrin.obj
 0001:00017775       __FIsin                    00028775   libf:intrin.obj
 0001:0001778f       __FItan                    0002878f   libf:intrin.obj
 0001:000177a9       __FIsqrt                   000287a9   libf:intrin.obj
 0001:000177c3       __FIdprod                  000287c3   libf:intrin.obj
 0001:000177c6       __FIlog                    000287c6   libf:intrin.obj
 0001:000177e0       __FIalog10                 000287e0   libf:intrin.obj
 0001:000177fa       __FIacos                   000287fa   libf:intrin.obj
 0001:00017814       __FIcosh                   00028814   libf:intrin.obj
 0001:0001782e       __FIasin                   0002882e   libf:intrin.obj
 0001:00017848       __FIsinh                   00028848   libf:intrin.obj
 0001:00017862       __FIatan                   00028862   libf:intrin.obj
 0001:0001787c       __FIatan2                  0002887c   libf:intrin.obj
 0001:00017896       __FItanh                   00028896   libf:intrin.obj
 0001:000178b0       __FIcotan                  000288b0   libf:intrin.obj
 0001:000178e0       __FIexp                    000288e0   libf:intrin.obj
 0001:000178fa       __FIamod                   000288fa   libf:intrin.obj
 0001:00017914       __FIsign                   00028914   libf:intrin.obj
 0001:00017948       __FIdim                    00028948   libf:intrin.obj
 0001:00017981       __FIaint                   00028981   libf:intrin.obj
 0001:00017981       __FIIaint                  00028981   libf:intrin.obj
 0001:000179a8       __FIanint                  000289a8   libf:intrin.obj
 0001:000179a8       __FIIanint                 000289a8   libf:intrin.obj
 0001:00017a11       __FIIcdiv                  00028a11   libf:intrin.obj
 0001:00017a11       __FIcdiv                   00028a11   libf:intrin.obj
 0001:00017b0d       __FIcpow                   00028b0d   libf:intrin.obj
 0001:00017c03       __FIcabs                   00028c03   libf:intrin.obj
 0001:00017c77       __FIccos                   00028c77   libf:intrin.obj
 0001:00017ce0       __FIcsin                   00028ce0   libf:intrin.obj
 0001:00017d47       __FIcexp                   00028d47   libf:intrin.obj
 0001:00017d98       __FIclog                   00028d98   libf:intrin.obj
 0001:00017dec       __FIcsqrt                  00028dec   libf:intrin.obj
 0001:00017ea0       __chkstk                   00028ea0   libf:chkstk.obj
 0001:00017f00       __setvideomoderows         00028f00   libf:qcsetmod.obj
 0001:00017f1d       __setvideomode             00028f1d   libf:qcsetmod.obj
 0001:00018092       __settextrows              00029092   libf:qcsetmod.obj
 0001:00018102       _$_init_max                00029102   libf:qcsetmod.obj
 0001:00018180       ___FF_hex@0                00029180 f libf:hex.obj
 0001:00018360       __FFuio                    00029360 f libf:uio.obj
 0001:00018630       ___FF_bino@4               00029630 f libf:bino.obj
 0001:00018790       ___FF_nrecini@0            00029790 f libf:nrecini.obj
 0001:000187b0       ___FF_bini@4               000297b0 f libf:bini.obj
 0001:00018870       ___FF_ufseqo@4             00029870 f libf:ufseqo.obj
 0001:00018a90       ___FF_ufdiri@4             00029a90 f libf:ufdiri.obj
 0001:00018ba0       _gettok@0                  00029ba0 f libf:fmtcr.obj
 0001:00018c90       _putint@4                  00029c90 f libf:fmtcr.obj
 0001:00018cd0       _copyint@0                 00029cd0 f libf:fmtcr.obj
 0001:00018d00       __FFfmtcr                  00029d00 f libf:fmtcr.obj
 0001:00019360       ___FF_putbint@8            0002a360 f libf:tab.obj
 0001:00019530       ___FF_inrepo@4             0002a530 f libf:tab.obj
 0001:00019640       ___FF_getnumt@0            0002a640 f libf:tab.obj
 0001:00019700       ___FF_getchnt@0            0002a700 f libf:tab.obj
 0001:000197a0       __FFwr2                    0002a7a0 f libf:wr2.obj
 0001:00019800       ___FF_ufdiro@4             0002a800 f libf:ufdiro.obj
 0001:000198e0       ___FF_ufseqi@4             0002a8e0 f libf:ufseqi.obj
 0001:00019aa0       ___FHvexpl@8               0002aaa0 f libf:helper.obj
 0001:00019b20       ___FHfexpl@8               0002ab20 f libf:helper.obj
 0001:00019b60       ___FHishal@8               0002ab60 f libf:helper.obj
 0001:00019bb0       ___FHishll@8               0002abb0 f libf:helper.obj
 0001:00019bf0       ___FHlink@4                0002abf0 f libf:helper.obj
 0001:00019c10       ___FHunlink@0              0002ac10 f libf:helper.obj
 0001:00019c20       ___FHbigint@0              0002ac20 f libf:helper.obj
 0001:00019c40       ___FHranger@0              0002ac40 f libf:helper.obj
 0001:00019c60       ___FHsranger@0             0002ac60 f libf:helper.obj
 0001:00019c80       ___FHAGOTO@0               0002ac80 f libf:helper.obj
 0001:00019ca0       ___FHovfl@0                0002aca0 f libf:helper.obj
 0001:00019cc0       ___FHCASE@0                0002acc0 f libf:helper.obj
 0001:00019ce0       ___Dollar_debug_unwind     0002ace0 f libf:helper.obj
 0001:00019ebb       _GetTimeZoneInformation@4  0002aebb f libf:fhack.obj
 0001:00019f59       _OpenProcessToken@12       0002af59 f libf:fhack.obj
 0001:00019fc3       _AdjustTokenPrivileges@24  0002afc3 f libf:fhack.obj
 0001:0001a039       _LookupPrivilegeValueA@12  0002b039 f libf:fhack.obj
 0001:0001a0a3       _GETCHARQQ@8               0002b0a3 f libf:fhack.obj
 0001:0001a0f8       _PEEKCHARQQ@0              0002b0f8 f libf:fhack.obj
 0001:0001a18c       _GETSTRQQ@8                0002b18c f libf:fhack.obj
 0001:0001a3c0       _NARGS@0                   0002b3c0 f libf:args.obj
 0001:0001a3d0       _GETARG@16                 0002b3d0 f libf:args.obj
 0001:0001a460       _GETTIM@16                 0002b460 f libf:timdat.obj
 0001:0001a4b0       _GETDAT@12                 0002b4b0 f libf:timdat.obj
 0001:0001a4f0       _SETTIM@16                 0002b4f0 f libf:timdat.obj
 0001:0001a5c0       _SETDAT@12                 0002b5c0 f libf:timdat.obj
 0001:0001a680       __FFpPAUSE                 0002b680 f libf:ppause.obj
 0001:0001a6f0       _GETFILEINFOQQ@16          0002b6f0 f libf:files.obj
 0001:0001a850       _BadInfo                   0002b850 f libf:files.obj
 0001:0001a890       _CopyInfo                  0002b890 f libf:files.obj
 0001:0001a8e0       _SETFILETIMEQQ@12          0002b8e0 f libf:files.obj
 0001:0001a970       _SETFILEACCESSQQ@12        0002b970 f libf:files.obj
 0001:0001a9f0       _RENAMEFILEQQ@16           0002b9f0 f libf:files.obj
 0001:0001aa90       _DELFILESQQ@8              0002ba90 f libf:files.obj
 0001:0001ab70       _FINDFILEQQ@24             0002bb70 f libf:files.obj
 0001:0001ac70       _PACKTIMEQQ@28             0002bc70 f libf:files.obj
 0001:0001ad00       _UNPACKTIMEQQ@28           0002bd00 f libf:files.obj
 0001:0001adbc       __getimage                 0002bdbc   libf:qcimage.obj
 0001:0001aebe       __putimage                 0002bebe   libf:qcimage.obj
 0001:0001afa5       __imagesize                0002bfa5   libf:qcimage.obj
 0001:0001b010       __setactivepage            0002c010   libf:qcpage.obj
 0001:0001b04f       __setvisualpage            0002c04f   libf:qcpage.obj
 0001:0001b08e       __getactivepage            0002c08e   libf:qcpage.obj
 0001:0001b09c       __getvisualpage            0002c09c   libf:qcpage.obj
 0001:0001b0b0       __setcolor                 0002c0b0   libf:qcpen.obj
 0001:0001b0df       __getcolor                 0002c0df   libf:qcpen.obj
 0001:0001b100       __setlinestyle             0002c100   libf:qcpen.obj
 0001:0001b129       __getlinestyle             0002c129   libf:qcpen.obj
 0001:0001b142       __remappalette             0002c142   libf:qcpen.obj
 0001:0001b27e       __remapallpalette          0002c27e   libf:qcpen.obj
 0001:0001b2cc       __selectpalette            0002c2cc   libf:qcpen.obj
 0001:0001b300       _GFStrToCStr@12            0002c300 f libf:stub.obj
 0001:0001b364       __f_settextposition@12     0002c364 f libf:stub.obj
 0001:0001b388       __f_gettextposition@4      0002c388 f libf:stub.obj
 0001:0001b39c       __f_outtext@8              0002c39c f libf:stub.obj
 0001:0001b3c8       __f_outmem@8               0002c3c8 f libf:stub.obj
 0001:0001b3dc       __f_getcurrentposition@4   0002c3dc f libf:stub.obj
 0001:0001b3fc       __f_moveto@12              0002c3fc f libf:stub.obj
 0001:0001b430       __f_setwindow@20           0002c430 f libf:stub.obj
 0001:0001b468       __f_getphyscoord@12        0002c468 f libf:stub.obj
 0001:0001b49c       __f_getviewcoord@12        0002c49c f libf:stub.obj
 0001:0001b4d0       __f_setvieworg@12          0002c4d0 f libf:stub.obj
 0001:0001b504       __f_getwindowcoord@12      0002c504 f libf:stub.obj
 0001:0001b538       __f_getviewcoord_w@12      0002c538 f libf:stub.obj
 0001:0001b56c       __f_getcurrentposition_wxy@4 0002c56c f libf:stub.obj
 0001:0001b590       __f_moveto_w@12            0002c590 f libf:stub.obj
 0001:0001b5c4       __f_registerfonts@8        0002c5c4 f libf:stub.obj
 0001:0001b608       __f_setfont@8              0002c608 f libf:stub.obj
 0001:0001b64c       __f_getfontinfo@4          0002c64c f libf:stub.obj
 0001:0001b694       __f_outgtext@8             0002c694 f libf:stub.obj
 0001:0001b6c0       __f_getgtextextent@8       0002c6c0 f libf:stub.obj
 0001:0001b6f4       __f_getgtextvector@8       0002c6f4 f libf:stub.obj
 0001:0001b71c       __f_loadimage@16           0002c71c f libf:stub.obj
 0001:0001b76c       __f_saveimage@24           0002c76c f libf:stub.obj
 0001:0001b7cc       __f_loadimage_w@16         0002c7cc f libf:stub.obj
 0001:0001b820       __f_saveimage_w@24         0002c820 f libf:stub.obj
 0001:0001b890       __settextcolor             0002c890   libf:qctxtcol.obj
 0001:0001b8b0       __gettextcolor             0002c8b0   libf:qctxtcol.obj
 0001:0001b8c0       _B$ScreenInit              0002c8c0   libf:llinit.obj
 0001:0001b987       _B$SetAdapter              0002c987   libf:llinit.obj
 0001:0001bc47       _B$ChkVGA                  0002cc47   libf:llinit.obj
 0001:0001bc6e       _B$ChkMonitor              0002cc6e   libf:llinit.obj
 0001:0001bcc0       __grstatus                 0002ccc0   libf:qcinit.obj
 0001:0001bcc8       _$_SetRows                 0002ccc8   libf:qcinit.obj
 0001:0001bd0b       _$_ChkRows                 0002cd0b   libf:qcinit.obj
 0001:0001bd78       _$_FixMaxPage              0002cd78   libf:qcinit.obj
 0001:0001bdb7       _$_init_mode               0002cdb7   libf:qcinit.obj
 0001:0001be5d       ___QCGINIT                 0002ce5d   libf:qcinit.obj
 0001:0001bf55       ___QCGTERM                 0002cf55   libf:qcinit.obj
 0001:0001bf90       _B$InitModeData            0002cf90   libf:llcgrp.obj
 0001:0001c015       _B$MapVWC                  0002d015   libf:llcgrp.obj
 0001:0001c0c4       _B$OutWord                 0002d0c4   libf:llcgrp.obj
 0001:0001c0cd       _B$ResetEGA                0002d0cd   libf:llcgrp.obj
 0001:0001c130       ___FF_puterr@12            0002d130 f libf:puterr.obj
 0001:0001c4a0       ___FF_error@8              0002d4a0 f libf:puterr.obj
 0001:0001c630       __arndfstr                 0002d630 f libf:arndfstr.obj
 0001:0001c6d0       ___FF_getname@4            0002d6d0 f libf:core.obj
 0001:0001c740       ___FF_xerrs@4              0002d740 f libf:core.obj
 0001:0001c780       __FFend                    0002d780 f libf:core.obj
 0001:0001c890       __FFinit                   0002d890 f libf:core.obj
 0001:0001c9e0       __FFinit_dll               0002d9e0 f libf:core.obj
 0001:0001cb20       ___FF_rmblanks@0           0002db20 f libf:core.obj
 0001:0001cb70       ___FFtk@12                 0002db70 f libf:core.obj
 0001:0001cd00       ___FFgn@0                  0002dd00 f libf:core.obj
 0001:0001cd10       ___FF_findrec@4            0002dd10 f libf:core.obj
 0001:0001cd90       ___FFpu@4                  0002dd90 f libf:core.obj
 0001:0001cf00       ___FF_searchunit@4         0002df00 f libf:core.obj
 0001:0001cfc0       ___FF_searchfile@0         0002dfc0 f libf:core.obj
 0001:0001d070       ___FF_getfip@4             0002e070 f libf:core.obj
 0001:0001d0e0       ___FFio@12                 0002e0e0 f libf:core.obj
 0001:0001d160       ___FF_isdevice@0           0002e160 f libf:core.obj
 0001:0001d250       ___FF_op@8                 0002e250 f libf:core.obj
 0001:0001d7e0       ___FF_werr@0               0002e7e0 f libf:core.obj
 0001:0001d820       ___FF_flushbuf@8           0002e820 f libf:core.obj
 0001:0001d960       ___FF_chw2r@0              0002e960 f libf:core.obj
 0001:0001d9e0       ___FF_cl@12                0002e9e0 f libf:core.obj
 0001:0001db90       ___FF_freefcb@12           0002eb90 f libf:core.obj
 0001:0001dc80       ___FF_chtmod@0             0002ec80 f libf:core.obj
 0001:0001dcb0       ___FF_oread@8              0002ecb0 f libf:core.obj
 0001:0001ddd0       ___FF_owrite@4             0002edd0 f libf:core.obj
 0001:0001de00       ___FF_alloc@4              0002ee00 f libf:core.obj
 0001:0001de30       ___FF_getfcb@4             0002ee30 f libf:core.obj
 0001:0001dec0       ___FF_putds@8              0002eec0 f libf:core.obj
 0001:0001df10       __FFStubFunc@0             0002ef10 f libf:core.obj
 0001:0001df20       _IsWindows                 0002ef20 f libf:core.obj
 0001:0001df50       _InitNullP                 0002ef50 f libf:core.obj
 0001:0001df70       _CheckNullP                0002ef70 f libf:core.obj
 0001:0001dfa0       _RError                    0002efa0 f libf:core.obj
 0001:0001dff0       _GetStackSize              0002eff0 f libf:core.obj
 0001:0001e000       ___FFgi@4                  0002f000 f libf:gi.obj
 0001:0001e090       ___FFgm@8                  0002f090 f libf:getitem.obj
 0001:0001e1a0       ___FFgs@12                 0002f1a0 f libf:getitem.obj
 0001:0001e1e0       ___FF_getitem@4            0002f1e0 f libf:getitem.obj
 0001:0001e2e0       ___FF_intin@4              0002f2e0 f libf:intin.obj
 0001:0001e350       ___FF_fillbuf@0            0002f350 f libf:fillbuf.obj
 0001:0001e550       ___FF_output@0             0002f550 f libf:output.obj
 0001:0001e770       ___FF_input@0              0002f770 f libf:input.obj
 0001:0001eb30       ___FF_getred@4             0002fb30 f libf:getred.obj
 0001:0001eff0       ___FF_nrecfdo@0            0002fff0   libf:iodec2.obj
 0001:0001eff0       ___FF_nrecfdi@0            0002fff0   libf:iodec2.obj
 0001:0001eff0       _stub0@0                   0002fff0   libf:iodec2.obj
 0001:0001eff3       ___FF_nlin@4               0002fff3   libf:iodec2.obj
 0001:0001eff3       _stub1@4                   0002fff3   libf:iodec2.obj
 0001:0001eff3       ___FF_nlout@4              0002fff3   libf:iodec2.obj
 0001:0001effc       _stub2@8                   0002fffc   libf:iodec2.obj
 0001:0001f010       ___FF_putbin@8             00030010 f libf:putbin.obj
 0001:0001f0e0       ___FF_getlong@0            000300e0 f libf:putbin.obj
 0001:0001f140       ___FF_getnum@0             00030140 f libf:getnum.obj
 0001:0001f420       ___FF_trunc@0              00030420 f libf:trunc.obj
 0001:0001f480       ___FF_crkrw@0              00030480 f libf:crkrw.obj
 0001:0001f710       _FStrToCStr@12             00030710 f libf:miscproc.obj
 0001:0001f780       _CStrToFStr@16             00030780 f libf:miscproc.obj
 0001:0001f7f0       _GETLASTERRORQQ@0          000307f0 f libf:miscproc.obj
 0001:0001f800       _SETERRORMODEQQ@4          00030800 f libf:miscproc.obj
 0001:0001f840       _GETENVQQ@16               00030840 f libf:miscproc.obj
 0001:0001f8d0       _SETENVQQ@8                000308d0 f libf:miscproc.obj
 0001:0001f990       _SLEEPQQ@4                 00030990 f libf:miscproc.obj
 0001:0001f9a0       _BEEPQQ@8                  000309a0 f libf:miscproc.obj
 0001:0001f9c0       _GETCONFIGQQ@0             000309c0 f libf:miscproc.obj
 0001:0001f9d0       ___FF_strtol@8             000309d0 f libf:fstrtol.obj
 0001:0001fbc0       ___FF_converchar@4         00030bc0 f libf:fstrtol.obj
 0001:0001fc10       ___FF_cctl@4               00030c10 f libf:cctl.obj
 0001:0001fc80       __matherr                  00030c80 f libf:matherr.obj
 0001:000200d0       _GetFpArgs                 000310d0 f libf:matherr.obj
 0001:00020150       _SetFpReturn               00031150 f libf:matherr.obj
 0001:000201f0       ___FF_mputerr              000311f0 f libf:matherr.obj
 0001:000205f0       _FixMathExceptions         000315f0 f libf:matherr.obj
 0001:00020620       _MathSignal                00031620 f libf:matherr.obj
 0001:00020660       _InIntrinsic               00031660 f libf:matherr.obj
 0001:000206b0       _$_qcg_enter               000316b0   libf:qccore.obj
 0001:000206e7       _$_qcg_exit                000316e7   libf:qccore.obj
 0001:000208ff       _$_home_cursor             000318ff   libf:qccore.obj
 0001:0002090f       _$_text_set_cursor         0003190f   libf:qccore.obj
 0001:0002093e       _$_set_color               0003193e   libf:qccore.obj
 0001:0002096b       _$_set_bk_color            0003196b   libf:qccore.obj
 0001:00020a1b       _$_set_text_color          00031a1b   libf:qccore.obj
 0001:00020a50       _$_set_text_attrib         00031a50   libf:qccore.obj
 0001:00020a98       _$_select_palette          00031a98   libf:qccore.obj
 0001:00020b7a       _$_limit                   00031b7a   libf:qccore.obj
 0001:00020b9b       _$_update_text_cursor      00031b9b   libf:qccore.obj
 0001:00020bcc       _$_unmap_cursor            00031bcc   libf:qccore.obj
 0001:00020bfb       _$_map_cursor              00031bfb   libf:qccore.obj
 0001:00020c73       _$_scroll                  00031c73   libf:qccore.obj
 0001:00020cb0       _B$SCNIO                   00031cb0   libf:llcscn.obj
 0001:00020cbf       _B$GrScreenSize            00031cbf   libf:llcscn.obj
 0001:00020cd2       _B$GRMODE                  00031cd2   libf:llcscn.obj
 0001:00020cda       _B$SELVPG                  00031cda   libf:llcscn.obj
 0001:00020ce1       _B$SELAPG                  00031ce1   libf:llcscn.obj
 0001:00020d13       _B$GETCSRDATA              00031d13   libf:llcscn.obj
 0001:00020d76       _B$OVWCSR                  00031d76   libf:llcscn.obj
 0001:00020d7e       _B$OFFCSR                  00031d7e   libf:llcscn.obj
 0001:00020d82       _B$CSRDSP                  00031d82   libf:llcscn.obj
 0001:00020de1       _B$ErrorReturn             00031de1   libf:llcscn.obj
 0001:00020df0       _GetDosBlock               00031df0   libf:dosx.obj
 0001:00020e09       _FreeDosBlock              00031e09   libf:dosx.obj
 0001:00020e23       _B$NearRet                 00031e23   libf:dosx.obj
 0001:00020e24       _$_EnsScrSwap              00031e24   libf:dosx.obj
 0001:00020e25       _SCNDIR                    00031e25   libf:dosx.obj
 0001:00020e26       _B$FarRet                  00031e26   libf:dosx.obj
 0001:00020e27       _B$InitSelTable            00031e27   libf:dosx.obj
 0001:0002101d       _B$Screen11                0003201d   libf:llvga.obj
 0001:00021051       _B$Screen12                00032051   libf:llvga.obj
 0001:00021073       _B$Screen13                00032073   libf:llvga.obj
 0001:0002108c       _B$Screen102               0003208c   libf:llvga.obj
 0001:000210d0       _$_VgaChkRows              000320d0   libf:llvga.obj
 0001:0002113d       _B$VgaSetPages             0003213d   libf:llvga.obj
 0001:00021150       _B$Vga256PalReset          00032150   libf:llvga.obj
 0001:00021157       _B$VgaPalReset             00032157   libf:llvga.obj
 0001:000211a9       _B$VgaPalPut               000321a9   libf:llvga.obj
 0001:000211da       _B$VgaPalTrans11           000321da   libf:llvga.obj
 0001:000211e6       _B$VgaPalTrans12           000321e6   libf:llvga.obj
 0001:000211eb       _B$VgaPalTrans13           000321eb   libf:llvga.obj
 0001:0002121a       _B$SetAttr256              0003221a   libf:llvga.obj
 0001:00021252       _B$VgaLineX256             00032252   libf:llvga.obj
 0001:0002130a       _B$VgaLineY256             0003230a   libf:llvga.obj
 0001:000213d2       _B$VgaLineV256             000323d2   libf:llvga.obj
 0001:0002147a       _B$VgaPutAction_13         0003247a   libf:llvga.obj
 0001:0002148e       _B$VgaWriteAction256       0003248e   libf:llvga.obj
 0001:0002149a       _B$VgaNReadL_13            0003249a   libf:llvga.obj
 0001:000214a7       _B$VgaNWriteL_13           000324a7   libf:llvga.obj
 0001:000214d7       _B$VgaNSetC_13             000324d7   libf:llvga.obj
 0001:00021529       _B$VgaScanL256             00032529   libf:llvga.obj
 0001:0002163b       _B$INIT_BKG_MASK13         0003263b   libf:llvga.obj
 0001:00021806       _b$SimVesaWinFunc          00032806   libf:llvesa.obj
 0001:00021844       _B$ChkVESA                 00032844   libf:llvesa.obj
 0001:0002192e       _B$Screen10X               0003292e   libf:llvesa.obj
 0001:00021c14       _$_VesaInitMaxColor        00032c14   libf:llvesa.obj
 0001:00021d6a       _B$SetVesaWinChk           00032d6a   libf:llvesa.obj
 0001:00021d7a       _B$ResetVESA               00032d7a   libf:llvesa.obj
 0001:00021dbf       _B$SetVesaWin              00032dbf   libf:llvesa.obj
 0001:00021e1a       _B$DecPageC                00032e1a   libf:llvesa.obj
 0001:00021e2e       _B$IncPageC                00032e2e   libf:llvesa.obj
 0001:00021e95       _VesaChkDownC              00032e95   libf:llvesa.obj
 0001:00021ebe       _VesaDownC                 00032ebe   libf:llvesa.obj
 0001:00021f97       _B$DecVesaWin              00032f97   libf:llvesa.obj
 0001:00021fa3       _B$IncVesaWin              00032fa3   libf:llvesa.obj
 0001:00021fb8       _VesaNReadL256             00032fb8   libf:llvesa.obj
 0001:00021fe0       _VesaNReadL256a            00032fe0   libf:llvesa.obj
 0001:00022068       _VesaNWriteL256a           00033068   libf:llvesa.obj
 0001:00022338       _B$VesaEgaScanLHelper      00033338   libf:llvesa.obj
 0001:00022377       _B$VesaEgaScanRHelper      00033377   libf:llvesa.obj
 0001:0002245f       _B$Screen4                 0003345f   libf:lloga.obj
 0001:000224c2       _B$ChkOlivetti             000334c2   libf:lloga.obj
 0001:00022550       __FFwrite                  00033550 f libf:ffwrite.obj
 0001:00022620       ___FF_getu_item@0          00033620 f libf:ugi.obj
 0001:00022680       __FFread                   00033680 f libf:ffread.obj
 0001:00022770       _$_coords                  00033770   libf:grputil.obj
 0001:0002279d       _B$INVIEW                  0003379d   libf:grputil.obj
 0001:000227d0       _B$PutGetInit              000337d0   libf:llagrp.obj
 0001:0002284a       _B$NReadC                  0003384a   libf:llagrp.obj
 0001:0002289c       _B$NWriteC                 0003389c   libf:llagrp.obj
 0001:000228f9       _B$PaintInit               000338f9   libf:llagrp.obj
 0001:00022934       _B$TileMod                 00033934   libf:llagrp.obj
 0001:00022943       _B$StoreC                  00033943   libf:llagrp.obj
 0001:00022959       _B$FetchC                  00033959   libf:llagrp.obj
 0001:00022970       _b$ColorPalette            00033970   libf:llxgasup.obj
 0001:00022980       _b$EnhPalette              00033980   libf:llxgasup.obj
 0001:0002299a       _B$EgaPalReset             0003399a   libf:llxgasup.obj
 0001:000229a3       _B$EgaPalResetB            000339a3   libf:llxgasup.obj
 0001:000229e3       _B$EgaPalPut               000339e3   libf:llxgasup.obj
 0001:000229ec       _B$EgaPalPutB              000339ec   libf:llxgasup.obj
 0001:00022a23       _B$EgaPalTrans             00033a23   libf:llxgasup.obj
 0001:00022a8d       _B$EgaPalSet               00033a8d   libf:llxgasup.obj
 0001:00022e50       __settextposition          00033e50   libf:qctxtpos.obj
 0001:00022e95       __gettextposition          00033e95   libf:qctxtpos.obj
 0001:00022ec0       _$_set_text_position       00033ec0   libf:qctxtpos.obj
 0001:00022f10       __outtext                  00033f10   libf:qctext.obj
 0001:00022f9d       __outmem                   00033f9d   libf:qctext.obj
 0001:00022ff7       __inchar                   00033ff7   libf:qctext.obj
 0001:000230ac       _$_scroll_window           000340ac   libf:qctext.obj
 0001:000230ea       _$_fix_text_position       000340ea   libf:qctext.obj
 0001:00023190       __setwritemode             00034190   libf:qcline.obj
 0001:000231c9       __getwritemode             000341c9   libf:qcline.obj
 0001:000231eb       __moveto                   000341eb   libf:qcline.obj
 0001:000231eb       __moveto_xy                000341eb   libf:qcline.obj
 0001:00023223       __getcurrentposition       00034223   libf:qcline.obj
 0001:00023246       __lineto                   00034246   libf:qcline.obj
 0001:00023246       __lineto_xy                00034246   libf:qcline.obj
 0001:0002332b       __getviewcoord_wxy         0003432b   libf:qcwindow.obj
 0001:0002334c       __getviewcoord_w           0003434c   libf:qcwindow.obj
 0001:00023371       _Map_WtoV                  00034371   libf:qcwindow.obj
 0001:0002339e       __getwindowcoord_xy        0003439e   libf:qcwindow.obj
 0001:0002339e       __getwindowcoord           0003439e   libf:qcwindow.obj
 0001:000233d4       __getcurrentposition_w     000343d4   libf:qcwindow.obj
 0001:0002340d       __setwindow                0003440d   libf:qcwindow.obj
 0001:000234c0       __setvieworg               000344c0   libf:qcview.obj
 0001:000234f9       __setcliprgn               000344f9   libf:qcview.obj
 0001:00023532       __setviewport              00034532   libf:qcview.obj
 0001:00023596       __getphyscoord             00034596   libf:qcview.obj
 0001:000235d0       __getviewcoord             000345d0   libf:qcview.obj
 0001:00023670       __moveto_w                 00034670   libf:qcline_w.obj
 0001:000236bd       __lineto_w                 000346bd   libf:qcline_w.obj
 0001:00023d70       __registerfonts            00034d70 f libf:fontlib.obj
 0001:00023ea4       __unregisterfonts          00034ea4 f libf:fontlib.obj
 0001:00023ef8       __setfont                  00034ef8 f libf:fontlib.obj
 0001:0002428c       __getfontinfo              0003528c f libf:fontlib.obj
 0001:000245ac       __outgtext                 000355ac f libf:fontlib.obj
 0001:000247a4       __getgtextextent           000357a4 f libf:fontlib.obj
 0001:000248e0       __setgtextvector           000358e0   libf:fontchar.obj
 0001:0002493f       __getgtextvector           0003593f   libf:fontchar.obj
 0001:00024956       __BltChar                  00035956   libf:fontchar.obj
 0001:00024aa0       _makeColorTable            00035aa0 f libf:dump.obj
 0001:00024b4c       _getIndex                  00035b4c f libf:dump.obj
 0001:00024b78       __saveimage                00035b78 f libf:dump.obj
 0001:00025044       __loadimage                00036044 f libf:dump.obj
 0001:00025760       __loadimage_w              00036760   libf:dump_w.obj
 0001:00025786       __loadimage_wxy            00036786   libf:dump_w.obj
 0001:000257ab       __saveimage_w              000367ab   libf:dump_w.obj
 0001:000257e5       __saveimage_wxy            000367e5   libf:dump_w.obj
 0001:00025820       _B$TntInit                 00036820 f libf:tntinit.obj
 0001:000258e4       _InitVESA1C                000368e4 f libf:tntinit.obj
 0001:0002591c       _SetZeroSeg                0003691c f libf:tntinit.obj
 0001:0002595c       _SetVideoSel               0003695c f libf:tntinit.obj
 0001:00025daa       _B$Screen7                 00036daa   libf:llega.obj
 0001:00025db1       _B$Screen8                 00036db1   libf:llega.obj
 0001:00025dc5       _B$Screen9                 00036dc5   libf:llega.obj
 0001:00025e0d       _B$Screen10                00036e0d   libf:llega.obj
 0001:00025e59       _B$EgaSetMode              00036e59   libf:llega.obj
 0001:00026390       _B$GRPINI                  00037390   libf:grinit.obj
 0001:000263e3       _B$VWINI                   000373e3   libf:grinit.obj
 0001:00026413       _B$VEWINI                  00037413   libf:grinit.obj
 0001:0002645e       _B$VWMAPC                  0003745e   libf:grinit.obj
 0001:000264a1       _B$GRPRST                  000374a1   libf:grinit.obj
 0001:000265da       _B$Mode0                   000375da   libf:lltext.obj
 0001:000265f2       _B$Mode1                   000375f2   libf:lltext.obj
 0001:000265f8       _B$Mode2                   000375f8   libf:lltext.obj
 0001:00026603       _B$Mode3                   00037603   libf:lltext.obj
 0001:00026609       _B$Mode7                   00037609   libf:lltext.obj
 0001:00026620       _B$FixTextPage             00037620   libf:lltext.obj
 0001:0002688e       _B$Mode5                   0003788e   libf:llcga.obj
 0001:00026894       _B$Mode4                   00037894   libf:llcga.obj
 0001:000268ef       _B$Screen2                 000378ef   libf:llcga.obj
 0001:00026b0f       _B$Screen3                 00037b0f   libf:llhgc.obj
 0001:00026be0       __FRerror@4                00037be0 f libf:build.obj
 0001:00026d30       ___FF_dbgmsg@0             00037d30 f libf:dbgmsg.obj
 0001:00026df0       _MATHERRQQ@20              00037df0 f libf:mhandler.obj
 0001:00026e00       _B$CgaSetAttr              00037e00   libf:llcgasup.obj
 0001:00026e0b       _B$CgaSetPages             00037e0b   libf:llcgasup.obj
 0001:00026e1e       _B$MapXYC2                 00037e1e   libf:llcgasup.obj
 0001:00026e3c       _B$MapXYC2_4               00037e3c   libf:llcgasup.obj
 0001:00026e67       _B$CgaReadC                00037e67   libf:llcgasup.obj
 0001:00026e8a       _B$CgaSetC                 00037e8a   libf:llcgasup.obj
 0001:00026ea4       _B$CgaSetPixC              00037ea4   libf:llcgasup.obj
 0001:00026ec1       _B$CgaSetPixFirstC         00037ec1   libf:llcgasup.obj
 0001:00026ec8       _B$CgaSetPixLastC          00037ec8   libf:llcgasup.obj
 0001:00026ec9       _B$CgaPutAction            00037ec9   libf:llcgasup.obj
 0001:00026f11       _B$CgaNReadL               00037f11   libf:llcgasup.obj
 0001:00026f2f       _B$CgaNWriteL              00037f2f   libf:llcgasup.obj
 0001:00026f88       _B$CgaNSetC                00037f88   libf:llcgasup.obj
 0001:0002707d       _B$CgaSetTile              0003807d   libf:llcgasup.obj
 0001:000270fa       _B$CgaScanL                000380fa   libf:llcgasup.obj
 0001:000271b1       _B$CgaScanR                000381b1   libf:llcgasup.obj
 0001:0002731d       _B$CgaLineX                0003831d   libf:llcgasup.obj
 0001:000273df       _B$CgaLineY                000383df   libf:llcgasup.obj
 0001:00027451       _B$CgaLineV                00038451   libf:llcgasup.obj
 0001:000274c0       _B$EgaMapXYC_102           000384c0   libf:llegasup.obj
 0001:000274d6       _B$EgaMapXYC_D             000384d6   libf:llegasup.obj
 0001:000274e2       _B$EgaMapXYC               000384e2   libf:llegasup.obj
 0001:0002753f       _B$EgaLeftC                0003853f   libf:llegasup.obj
 0001:00027548       _B$EgaLeftC_13             00038548   libf:llegasup.obj
 0001:0002754f       _B$EgaChkUpC               0003854f   libf:llegasup.obj
 0001:00027585       _B$EgaUpC                  00038585   libf:llegasup.obj
 0001:00027594       _B$EgaChkDownC             00038594   libf:llegasup.obj
 0001:000275ca       _B$EgaDownC                000385ca   libf:llegasup.obj
 0001:000275d9       _B$EgaSetAttr              000385d9   libf:llegasup.obj
 0001:000275ef       _B$EgaReadC                000385ef   libf:llegasup.obj
 0001:0002762f       _B$EgaReadC_F              0003862f   libf:llegasup.obj
 0001:0002763d       _B$EgaReadC_64K            0003863d   libf:llegasup.obj
 0001:00027651       _B$EgaSetC                 00038651   libf:llegasup.obj
 0001:0002768c       _B$EgaSetPixC              0003868c   libf:llegasup.obj
 0001:000276a8       _B$EgaSetPixFirstC         000386a8   libf:llegasup.obj
 0001:000276c4       _B$EgaLineX                000386c4   libf:llegasup.obj
 0001:0002774a       _B$EgaLineY                0003874a   libf:llegasup.obj
 0001:000277c8       _B$EgaLineV                000387c8   libf:llegasup.obj
 0001:0002781d       _B$EgaPutAction_64K        0003881d   libf:llegasup.obj
 0001:00027821       _B$EgaPutAction_F          00038821   libf:llegasup.obj
 0001:00027825       _B$EgaPutAction            00038825   libf:llegasup.obj
 0001:0002785a       _B$EgaNReadL_F             0003885a   libf:llegasup.obj
 0001:0002785c       _B$EgaNReadL               0003885c   libf:llegasup.obj
 0001:0002789c       _B$EgaNWriteL_F            0003889c   libf:llegasup.obj
 0001:000278a2       _B$EgaNWriteL              000388a2   libf:llegasup.obj
 0001:0002794d       _B$EgaNSetC                0003894d   libf:llegasup.obj
 0001:00027a66       _B$EgaPaintBound           00038a66   libf:llegasup.obj
 0001:00027a6b       _B$EgaSetColorBits         00038a6b   libf:llegasup.obj
 0001:00027ac3       _B$EgaPaintBoundCom        00038ac3   libf:llegasup.obj
 0001:00027b19       _B$EgaSetTile              00038b19   libf:llegasup.obj
 0001:00027b3e       _B$EgaScanInit             00038b3e   libf:llegasup.obj
 0001:00027b70       _B$EgaPAINPX               00038b70   libf:llegasup.obj
 0001:00027c87       _B$EgaPIXCNT               00038c87   libf:llegasup.obj
 0001:00027c92       _B$EgaSETCMP               00038c92   libf:llegasup.obj
 0001:00027cb1       _B$EgaCHKBTR               00038cb1   libf:llegasup.obj
 0001:00027ccd       _B$EgaCHKBTL               00038ccd   libf:llegasup.obj
 0001:00027d2e       _B$EgaTILRGT               00038d2e   libf:llegasup.obj
 0001:00027e30       _B$EgaTILLFT               00038e30   libf:llegasup.obj
 0001:00027f6a       _B$EgaScanL                00038f6a   libf:llegasup.obj
 0001:000280a5       _B$EgaScanR                000390a5   libf:llegasup.obj
 0001:000281e0       __clearscreen              000391e0   libf:qcclrscn.obj
 0001:000282b0       _B$CgaLeftC2               000392b0   libf:llhgcsup.obj
 0001:000282b6       _B$CgaLeftC1               000392b6   libf:llhgcsup.obj
 0001:000282c6       _B$CgaChkUpC               000392c6   libf:llhgcsup.obj
 0001:000282e5       _B$CgaUpC                  000392e5   libf:llhgcsup.obj
 0001:00028301       _B$CgaChkDownC             00039301   libf:llhgcsup.obj
 0001:00028320       _B$CgaDownC                00039320   libf:llhgcsup.obj
 0001:0002833c       _B$CgaPaintBound           0003933c   libf:llhgcsup.obj
 0001:00028380       _B$FastOutStr              00039380   libf:llscnio.obj
 0001:00028440       _B$BOXNOF                  00039440   libf:grline.obj
 0001:00028490       _B$LINDRW                  00039490   libf:grline.obj
 0001:000286c0       _B$CLINE2                  000396c0   libf:grline.obj
 0001:000287f0       _B$FPGRINI                 000397f0   libf:grfpinit.obj
 0001:0002884f       _B$WNDINX                  0003984f   libf:grfpinit.obj
 0001:00028898       _B$MAPPX2                  00039898   libf:grfpinit.obj
 0001:000288aa       _B$MAPPY2                  000398aa   libf:grfpinit.obj
 0001:000288e2       _B$ISWNDW                  000398e2   libf:grfpinit.obj
 0001:00028900       _B$XYSAVE                  00039900   libf:grwindow.obj
 0001:0002890c       _B$XCHGF                   0003990c   libf:grwindow.obj
 0001:0002893b       _B$QCMAPLPY                0003993b   libf:grwindow.obj
 0001:00028960       _B$QCMAPLPX                00039960   libf:grwindow.obj
 0001:00028980       __ChrToAnsi                00039980   libf:fontmap.obj
 0001:000289a0       __setpixel_xy              000399a0   libf:qcgr.obj
 0001:000289a0       __setpixel                 000399a0   libf:qcgr.obj
 0001:00028a0d       __getpixel                 00039a0d   libf:qcgr.obj
 0001:00028a0d       __getpixel_xy              00039a0d   libf:qcgr.obj
 0001:00028a50       __getColorInfo             00039a50   libf:getcolor.obj
 0001:00028b10       _B$VWFILL                  00039b10   libf:vwclr.obj
 0001:00028b46       _B$DOBOXF                  00039b46   libf:vwclr.obj
 0001:00028b65       _B$SCNFILL                 00039b65   libf:vwclr.obj
 0001:00028c51       _B$CLIPCK                  00039c51   libf:vwclr.obj
 0001:00028cca       _B$XDELT                   00039cca   libf:vwclr.obj
 0001:00028cda       _B$YDELT                   00039cda   libf:vwclr.obj
 0001:00028cf0       __OemToAnsiTable           00039cf0   libf:cp850.obj
 0001:00028d70       _mainCRTStartup            00039d70 f libc:CRT0.OBJ
 0001:00028e80       __amsg_exit                00039e80 f libc:CRT0.OBJ
 0001:00028eb0       __ftol                     00039eb0   libc:ftol.obj
 0001:00028ee0       __fpmath                   00039ee0 f libc:fpinit.obj
 0001:00028ef0       __fpclear                  00039ef0 f libc:fpinit.obj
 0001:00028f00       __cfltcvt_init             00039f00 f libc:fpinit.obj
 0001:00028f40       ___setfflag                00039f40 f libc:fpinit.obj
 0001:00028f50       _free                      00039f50 f libc:FREE.OBJ
 0001:00028fb0       _realloc                   00039fb0 f libc:REALLOC.OBJ
 0001:000290c0       __expand                   0003a0c0 f libc:REALLOC.OBJ
 0001:00029260       _malloc                    0003a260 f libc:MALLOC.OBJ
 0001:00029310       __heap_split_block         0003a310 f libc:MALLOC.OBJ
 0001:00029370       _memmove                   0003a370   libc:MEMMOVE.OBJ
 0001:000294c0       _memchr                    0003a4c0   libc:MEMCHR.OBJ
 0001:000294f0       __fltout                   0003a4f0 f libc:cfout.obj
 0001:00029560       ___dtold                   0003a560 f libc:cfout.obj
 0001:00029640       __cinit                    0003a640 f libc:CRT0DAT.OBJ
 0001:00029670       _exit                      0003a670 f libc:CRT0DAT.OBJ
 0001:00029690       __exit                     0003a690 f libc:CRT0DAT.OBJ
 0001:000296b0       __cexit                    0003a6b0 f libc:CRT0DAT.OBJ
 0001:000296c0       __c_exit                   0003a6c0 f libc:CRT0DAT.OBJ
 0001:00029780       __mktemp                   0003a780 f libc:MKTEMP.OBJ
 0001:00029850       __setjmp                   0003a850   libc:SETJMP.OBJ
 0001:0002988f       _longjmp                   0003a88f   libc:SETJMP.OBJ
 0001:000298e5       _raisex                    0003a8e5   libc:SETJMP.OBJ
 0001:00029920       __access                   0003a920 f libc:ACCESS.OBJ
 0001:00029970       __fltinf                   0003a970 f libc:fltinf.obj
 0001:00029a40       __isatty                   0003aa40 f libc:ISATTY.OBJ
 0001:00029ad0       __itoa                     0003aad0 f libc:XTOA.OBJ
 0001:00029b10       __ltoa                     0003ab10 f libc:XTOA.OBJ
 0001:00029b40       __ultoa                    0003ab40 f libc:XTOA.OBJ
 0001:00029b60       __spawnvpe                 0003ab60 f libc:SPAWNVPE.OBJ
 0001:00029cf0       _strtok                    0003acf0 f libc:STRTOK.OBJ
 0001:00029dd0       _system                    0003add0 f libc:SYSTEM.OBJ
 0001:00029e80       _sin                       0003ae80   libc:87ctrig.obj
 0001:00029e8a       _cos                       0003ae8a   libc:87ctrig.obj
 0001:00029e91       _tan                       0003ae91   libc:87ctrig.obj
 0001:00029e98       __CIsin                    0003ae98   libc:87ctrig.obj
 0001:00029ea2       __CIcos                    0003aea2   libc:87ctrig.obj
 0001:00029ea9       __CItan                    0003aea9   libc:87ctrig.obj
 0001:00029eb0       _sinh                      0003aeb0   libc:87ctrigh.obj
 0001:00029eba       _cosh                      0003aeba   libc:87ctrigh.obj
 0001:00029ec1       _tanh                      0003aec1   libc:87ctrigh.obj
 0001:00029ec8       __CIsinh                   0003aec8   libc:87ctrigh.obj
 0001:00029ed2       __CIcosh                   0003aed2   libc:87ctrigh.obj
 0001:00029ed9       __CItanh                   0003aed9   libc:87ctrigh.obj
 0001:00029ee0       _pow                       0003aee0   libc:87ctran.obj
 0001:00029eea       _log                       0003aeea   libc:87ctran.obj
 0001:00029ef4       _log10                     0003aef4   libc:87ctran.obj
 0001:00029efb       _exp                       0003aefb   libc:87ctran.obj
 0001:00029f02       __CIpow                    0003af02   libc:87ctran.obj
 0001:00029f0c       __CIlog                    0003af0c   libc:87ctran.obj
 0001:00029f16       __CIlog10                  0003af16   libc:87ctran.obj
 0001:00029f1d       __CIexp                    0003af1d   libc:87ctran.obj
 0001:00029f24       _asin                      0003af24   libc:87ctriga.obj
 0001:00029f2e       _acos                      0003af2e   libc:87ctriga.obj
 0001:00029f35       _atan                      0003af35   libc:87ctriga.obj
 0001:00029f3c       _atan2                     0003af3c   libc:87ctriga.obj
 0001:00029f46       __CIasin                   0003af46   libc:87ctriga.obj
 0001:00029f50       __CIacos                   0003af50   libc:87ctriga.obj
 0001:00029f57       __CIatan                   0003af57   libc:87ctriga.obj
 0001:00029f5e       __CIatan2                  0003af5e   libc:87ctriga.obj
 0001:00029f68       _sqrt                      0003af68   libc:87csqrt.obj
 0001:00029f72       __CIsqrt                   0003af72   libc:87csqrt.obj
 0001:00029f7c       _fmod                      0003af7c   libc:87fmod.obj
 0001:00029f86       __CIfmod                   0003af86   libc:87fmod.obj
 0001:00029fa0       __lseek                    0003afa0 f libc:LSEEK.OBJ
 0001:0002a020       _strchr                    0003b020   libc:STRCHR.OBJ
 0001:0002a050       ___tzset                   0003b050 f libc:TZSET.OBJ
 0001:0002a070       __tzset                    0003b070 f libc:TZSET.OBJ
 0001:0002a270       __isindst                  0003b270 f libc:TZSET.OBJ
 0001:0002a340       _getenv                    0003b340 f libc:GETENV.OBJ
 0001:0002a3c0       _memset                    0003b3c0   libc:MEMSET.OBJ
 0001:0002a410       __getch                    0003b410 f libc:GETCH.OBJ
 0001:0002a4f0       __getche                   0003b4f0 f libc:GETCH.OBJ
 0001:0002a520       __kbhit                    0003b520 f libc:GETCH.OBJ
 0001:0002a620       __ungetch                  0003b620 f libc:GETCH.OBJ
 0001:0002a750       __cputs                    0003b750 f libc:CPUTS.OBJ
 0001:0002a7a0       __cgets                    0003b7a0 f libc:CGETS.OBJ
 0001:0002a890       __findfirst                0003b890 f libc:FINDFILE.OBJ
 0001:0002a9c0       __findnext                 0003b9c0 f libc:FINDFILE.OBJ
 0001:0002aaf0       __findclose                0003baf0 f libc:FINDFILE.OBJ
 0001:0002aba0       __utime                    0003bba0 f libc:UTIME.OBJ
 0001:0002abe0       __futime                   0003bbe0 f libc:UTIME.OBJ
 0001:0002ad60       _rename                    0003bd60 f libc:RENAME.OBJ
 0001:0002ada0       _remove                    0003bda0 f libc:UNLINK.OBJ
 0001:0002add0       __unlink                   0003bdd0 f libc:UNLINK.OBJ
 0001:0002ade0       __searchenv                0003bde0 f libc:SEARCHEN.OBJ
 0001:0002af00       _mktime                    0003bf00 f libc:MKTIME.OBJ
 0001:0002af10       __mkgmtime                 0003bf10 f libc:MKTIME.OBJ
 0001:0002b180       _localtime                 0003c180 f libc:LOCALTIM.OBJ
 0001:0002b330       _strncpy                   0003c330   libc:STRNCPY.OBJ
 0001:0002b360       __onexit                   0003c360 f libc:ONEXIT.OBJ
 0001:0002b3e0       _atexit                    0003c3e0 f libc:ONEXIT.OBJ
 0001:0002b400       __onexitinit               0003c400 f libc:ONEXIT.OBJ
 0001:0002b440       __FF_MSGBANNER             0003c440 f libc:CRT0MSG.OBJ
 0001:0002b470       __NMSG_WRITE               0003c470 f libc:CRT0MSG.OBJ
 0001:0002b4d0       __GET_RTERRMSG             0003c4d0 f libc:CRT0MSG.OBJ
 0001:0002b510       __stricmp                  0003c510   libc:STRICMP.OBJ
 0001:0002b510       __strcmpi                  0003c510   libc:STRICMP.OBJ
 0001:0002b560       __fullpath                 0003c560 f libc:FULLPATH.OBJ
 0001:0002b8a0       __open                     0003c8a0 f libc:OPEN.OBJ
 0001:0002b8c0       __sopen                    0003c8c0 f libc:OPEN.OBJ
 0001:0002bcc0       __close                    0003ccc0 f libc:CLOSE.OBJ
 0001:0002bd60       __write                    0003cd60 f libc:WRITE.OBJ
 0001:0002bf90       __toupper                  0003cf90 f libc:TOUPPER.OBJ
 0001:0002bfa0       _toupper                   0003cfa0 f libc:TOUPPER.OBJ
 0001:0002c110       __chsize                   0003d110 f libc:CHSIZE.OBJ
 0001:0002c260       __strupr                   0003d260   libc:STRUPR.OBJ
 0001:0002c290       __putenv                   0003d290 f libc:PUTENV.OBJ
 0001:0002c4b0       __tolower                  0003d4b0 f libc:TOLOWER.OBJ
 0001:0002c4c0       _tolower                   0003d4c0 f libc:TOLOWER.OBJ
 0001:0002c630       _strncmp                   0003d630   libc:STRNCMP.OBJ
 0001:0002c6c0       _signal                    0003d6c0 f libc:WINSIG.OBJ
 0001:0002c800       _raise                     0003d800 f libc:WINSIG.OBJ
 0001:0002c9a0       __setmode                  0003d9a0 f libc:SETMODE.OBJ
 0001:0002ca40       __read                     0003da40 f libc:READ.OBJ
 0001:0002cc60       _atol                      0003dc60 f libc:ATOX.OBJ
 0001:0002cd10       _atoi                      0003dd10 f libc:ATOX.OBJ
 0001:0002cd20       _puts                      0003dd20 f libc:PUTS.OBJ
 0001:0002cdb4       __except_handler2          0003ddb4   libc:EXSUP.OBJ
 0001:0002ce7f       __global_unwind2           0003de7f   libc:EXSUP.OBJ
 0001:0002ce9f       __unwind_handler           0003de9f   libc:EXSUP.OBJ
 0001:0002cec5       __local_unwind2            0003dec5   libc:EXSUP.OBJ
 0001:0002cf2b       __abnormal_termination     0003df2b   libc:EXSUP.OBJ
 0001:0002cf60       __XcptFilter               0003df60 f libc:WINXFLTR.OBJ
 0001:0002d0c0       __setenvp                  0003e0c0 f libc:STDENVP.OBJ
 0001:0002d190       __setargv                  0003e190 f libc:STDARGV.OBJ
 0001:0002d3b0       __ioinit                   0003e3b0 f libc:IOINIT.OBJ
 0001:0002d4a0       __heap_init                0003e4a0 f libc:HEAPINIT.OBJ
 0001:0002d4c0       __heap_term                0003e4c0 f libc:HEAPINIT.OBJ
 0001:0002d530       __heap_grow_emptylist      0003e530 f libc:HEAPINIT.OBJ
 0001:0002d590       __setdefaultprecision      0003e590 f libc:fp8.obj
 0001:0002d5b0       __forcdecpt                0003e5b0 f libc:cvt.obj
 0001:0002d620       __cropzeros                0003e620 f libc:cvt.obj
 0001:0002d680       __positive                 0003e680 f libc:cvt.obj
 0001:0002d6a0       __fassign                  0003e6a0 f libc:cvt.obj
 0001:0002d6d0       __cftoe                    0003e6d0 f libc:cvt.obj
 0001:0002d840       __cftof                    0003e840 f libc:cvt.obj
 0001:0002d970       __cftog                    0003e970 f libc:cvt.obj
 0001:0002da30       __cfltcvt                  0003ea30 f libc:cvt.obj
 0001:0002dad0       __heap_abort               0003ead0 f libc:HPABORT.OBJ
 0001:0002dae0       __heap_grow                0003eae0 f libc:HEAPGROW.OBJ
 0001:0002dbe0       __heap_grow_region         0003ebe0 f libc:HEAPGROW.OBJ
 0001:0002dca0       __heap_free_region         0003eca0 f libc:HEAPGROW.OBJ
 0001:0002dcf0       __heap_search              0003ecf0 f libc:HEAPSRCH.OBJ
 0001:0002de00       _$I10_OUTPUT               0003ee00 f libc:x10fout.obj
 0001:0002e1a0       __getpid                   0003f1a0 f libc:GETPID.OBJ
 0001:0002e1b0       __dosmaperr                0003f1b0 f libc:DOSMAP.OBJ
 0001:0002e230       __ZeroTail                 0003f230 f libc:intrncvt.obj
 0001:0002e2a0       __IncMan                   0003f2a0 f libc:intrncvt.obj
 0001:0002e310       __RoundMan                 0003f310 f libc:intrncvt.obj
 0001:0002e3c0       __CopyMan                  0003f3c0 f libc:intrncvt.obj
 0001:0002e3e0       __FillZeroMan              0003f3e0 f libc:intrncvt.obj
 0001:0002e400       __IsZeroMan                0003f400 f libc:intrncvt.obj
 0001:0002e420       __ShrMan                   0003f420 f libc:intrncvt.obj
 0001:0002e4d0       __ld12cvt                  0003f4d0 f libc:intrncvt.obj
 0001:0002e6a0       __ld12tod                  0003f6a0 f libc:intrncvt.obj
 0001:0002e6c0       __ld12tof                  0003f6c0 f libc:intrncvt.obj
 0001:0002e6e0       __ld12told                 0003f6e0 f libc:intrncvt.obj
 0001:0002e770       __atodbl                   0003f770 f libc:intrncvt.obj
 0001:0002e7b0       __atoldbl                  0003f7b0 f libc:intrncvt.obj
 0001:0002e7f0       __atoflt                   0003f7f0 f libc:intrncvt.obj
 0001:0002e830       ___strgtold12              0003f830 f libc:strgtold.obj
 0001:0002ef80       ___STRINGTOLD              0003ff80 f libc:strgtold.obj
 0001:0002f040       __spawnve                  00040040 f libc:SPAWNVE.OBJ
 0001:0002f270       __getpath                  00040270 f libc:GETPATH.OBJ
 0001:0002f2f0       __fFCOS                    000402f0   libc:87trig.obj
 0001:0002f2fa       __fFSIN                    000402fa   libc:87trig.obj
 0001:0002f31c       __cintrindisp2             0004031c   libc:87cdisp.obj
 0001:0002f355       __cintrindisp1             00040355   libc:87cdisp.obj
 0001:0002f386       __ctrandisp2               00040386   libc:87cdisp.obj
 0001:0002f4fe       __ctrandisp1               000404fe   libc:87cdisp.obj
 0001:0002f525       __fload                    00040525   libc:87cdisp.obj
 0001:0002f560       __fFSINH                   00040560   libc:87trigh.obj
 0001:0002f5b2       __fFCOSH                   000405b2   libc:87trigh.obj
 0001:0002f66d       __fFEXP                    0004066d   libc:87tran.obj
 0001:0002f6c4       __rtinfpopse               000406c4   libc:87tran.obj
 0001:0002f6c6       __rtinfnpopse              000406c6   libc:87tran.obj
 0001:0002f6d6       __fFLN                     000406d6   libc:87tran.obj
 0001:0002f78b       __rtinfpop                 0004078b   libc:87tran.obj
 0001:0002f78d       __rtinfnpop                0004078d   libc:87tran.obj
 0001:0002f7aa       __ffexpm1                  000407aa   libc:87tran.obj
 0001:0002f870       __fFATN2                   00040870   libc:87triga.obj
 0001:0002f8c0       __rtpiby2                  000408c0   libc:87triga.obj
 0001:0002f914       __trandisp1                00040914   libc:87disp.obj
 0001:0002f97f       __trandisp2                0004097f   libc:87disp.obj
 0001:0002fa0f       __rttospopde               00040a0f   libc:87disp.obj
 0001:0002fa14       __rttospop                 00040a14   libc:87disp.obj
 0001:0002fa16       __rtnospop                 00040a16   libc:87disp.obj
 0001:0002fa18       __rttosnpop                00040a18   libc:87disp.obj
 0001:0002fa19       __rtnospopde               00040a19   libc:87disp.obj
 0001:0002fa20       __rtzeropop                00040a20   libc:87disp.obj
 0001:0002fa22       __rtzeronpop               00040a22   libc:87disp.obj
 0001:0002fa27       __rtonepop                 00040a27   libc:87disp.obj
 0001:0002fa29       __rtonenpop                00040a29   libc:87disp.obj
 0001:0002fa2e       __tosnan1                  00040a2e   libc:87disp.obj
 0001:0002fa59       __nosnan2                  00040a59   libc:87disp.obj
 0001:0002fa5b       __tosnan2                  00040a5b   libc:87disp.obj
 0001:0002fa86       __nan2                     00040a86   libc:87disp.obj
 0001:0002fac8       __rtindfpop                00040ac8   libc:87disp.obj
 0001:0002faca       __rtindfnpop               00040aca   libc:87disp.obj
 0001:0002fadb       __rttosnpopde              00040adb   libc:87disp.obj
 0001:0002fae5       __rtchsifneg               00040ae5   libc:87disp.obj
 0001:0002faf0       __alloc_osfhnd             00040af0 f libc:OSFINFO.OBJ
 0001:0002fb30       __set_osfhnd               00040b30 f libc:OSFINFO.OBJ
 0001:0002fbc0       __free_osfhnd              00040bc0 f libc:OSFINFO.OBJ
 0001:0002fc30       __get_osfhandle            00040c30 f libc:OSFINFO.OBJ
 0001:0002fc70       __open_osfhandle           00040c70 f libc:OSFINFO.OBJ
 0001:0002fd10       __strdup                   00040d10   libc:STRDUP.OBJ
 0001:0002fd38       __strnicmp                 00040d38   libc:STRNICMP.OBJ
 0001:0002fd90       __putch                    00040d90 f libc:PUTCH.OBJ
 0001:0002fde0       ___gmtotime_t              00040de0 f libc:DTOXTIME.OBJ
 0001:0002fe70       _gmtime                    00040e70 f libc:GMTIME.OBJ
 0001:0002ffc0       _time                      00040fc0 f libc:TIME.OBJ
 0001:00030020       __getcwd                   00041020 f libc:GETCWD.OBJ
 0001:00030040       __getdcwd                  00041040 f libc:GETCWD.OBJ
 0001:00030150       __validdrive               00041150 f libc:GETCWD.OBJ
 0001:00030170       __msize                    00041170 f libc:MSIZE.OBJ
 0001:00030190       __getdrive                 00041190 f libc:DRIVE.OBJ
 0001:000301d0       __chdrive                  000411d0 f libc:DRIVE.OBJ
 0001:000302b0       __isctype                  000412b0 f libc:ISCTYPE.OBJ
 0001:00030370       __stbuf                    00041370 f libc:_SFTBUF.OBJ
 0001:00030410       __ftbuf                    00041410 f libc:_SFTBUF.OBJ
 0001:00030460       __flsbuf                   00041460 f libc:_FLSBUF.OBJ
 0001:00030590       _fwrite                    00041590 f libc:FWRITE.OBJ
 0001:00030700       __statusfp                 00041700 f libc:ieee87.obj
 0001:00030720       __clearfp                  00041720 f libc:ieee87.obj
 0001:00030740       __control87                00041740 f libc:ieee87.obj
 0001:00030780       __controlfp                00041780 f libc:ieee87.obj
 0001:000307a0       __fpreset                  000417a0 f libc:ieee87.obj
 0001:00030970       __fptrap                   00041970 f libc:CRT0FP.OBJ
 0001:00030980       __fptostr                  00041980 f libc:_FPTOSTR.OBJ
 0001:00030a10       __heapadd                  00041a10 f libc:HEAPADD.OBJ
 0001:00030a40       __heap_addblock            00041a40 f libc:HEAPADD.OBJ
 0001:00030cc0       ___addl                    00041cc0 f libc:mantold.obj
 0001:00030cf0       ___add_12                  00041cf0 f libc:mantold.obj
 0001:00030d60       ___shl_12                  00041d60 f libc:mantold.obj
 0001:00030db0       ___shr_12                  00041db0 f libc:mantold.obj
 0001:00030e00       ___mtold12                 00041e00 f libc:mantold.obj
 0001:00030ef0       ___ld12mul                 00041ef0 f libc:tenpow.obj
 0001:000311f0       ___multtenpow12            000421f0 f libc:tenpow.obj
 0001:00031270       __dospawn                  00042270 f libc:DOSPAWN.OBJ
 0001:000314c0       __cenvarg                  000424c0 f libc:CENVARG.OBJ
 0001:00031830       _strrchr                   00042830   libc:STRRCHR.OBJ
 0001:00031860       __87except                 00042860 f libc:87except.obj
 0001:00031990       __powhlp                   00042990 f libc:powhlp.obj
 0001:00031c00       __d_inttype                00042c00 f libc:powhlp.obj
 0001:00031c70       _strcat                    00042c70   libc:STRCAT.OBJ
 0001:00031c74       _strcpy                    00042c74   libc:STRCAT.OBJ
 0001:00031d08       _strlen                    00042d08   libc:STRLEN.OBJ
 0001:00031d60       __initcon                  00042d60 f libc:INITCON.OBJ
 0001:00031da0       __termcon                  00042da0 f libc:INITCON.OBJ
 0001:00031dd0       _fflush                    00042dd0 f libc:FFLUSH.OBJ
 0001:00031e20       __flush                    00042e20 f libc:FFLUSH.OBJ
 0001:00031e90       __flushall                 00042e90 f libc:FFLUSH.OBJ
 0001:00031f10       __endstdio                 00042f10 f libc:FFLUSH.OBJ
 0001:00031f30       __getbuf                   00042f30 f libc:_GETBUF.OBJ
 0001:00031f80       __heap_findaddr            00042f80 f libc:FINDADDR.OBJ
 0001:00032000       _calloc                    00043000 f libc:CALLOC.OBJ
 0001:00032040       __handle_qnan1             00043040 f libc:fpexcept.obj
 0001:000320b0       __handle_qnan2             000430b0 f libc:fpexcept.obj
 0001:00032130       __except1                  00043130 f libc:fpexcept.obj
 0001:00032200       __except2                  00043200 f libc:fpexcept.obj
 0001:00032300       __raise_exc                00043300 f libc:fpexcept.obj
 0001:00032690       __handle_exc               00043690 f libc:fpexcept.obj
 0001:00032960       __umatherr                 00043960 f libc:fpexcept.obj
 0001:00032a10       __set_errno                00043a10 f libc:fpexcept.obj
 0001:00032a70       __errcode                  00043a70 f libc:fpexcept.obj
 0001:00032ab0       __statfp                   00043ab0 f libc:fpctrl.obj
 0001:00032ad0       __clrfp                    00043ad0 f libc:fpctrl.obj
 0001:00032af0       __ctrlfp                   00043af0 f libc:fpctrl.obj
 0001:00032b30       __set_statfp               00043b30 f libc:fpctrl.obj
 0001:00032b90       __set_exp                  00043b90 f libc:util.obj
 0001:00032bd0       __get_exp                  00043bd0 f libc:util.obj
 0001:00032bf0       __add_exp                  00043bf0 f libc:util.obj
 0001:00032c20       __set_bexp                 00043c20 f libc:util.obj
 0001:00032c60       __sptype                   00043c60 f libc:util.obj
 0001:00032cd0       __decomp                   00043cd0 f libc:util.obj
 0001:00032de0       __frnd                     00043de0 f libc:frnd.obj
 0001:00032e00       __commit                   00043e00 f libc:COMMIT.OBJ
 0001:00032e60       __fcloseall                00043e60 f libc:CLOSEALL.OBJ
 0001:00032ea0       _fclose                    00043ea0 f libc:FCLOSE.OBJ
 0001:00032f10       __freebuf                  00043f10 f libc:_FREEBUF.OBJ
 0001:00032f50       _GetCommandLineA@0         00043f50   kernel32:kernel32.def
 0001:00032f56       _GetVersion@0              00043f56   kernel32:kernel32.def
 0001:00032f5c       _GetProcAddress@8          00043f5c   kernel32:kernel32.def
 0001:00032f62       _LoadLibraryA@4            00043f62   kernel32:kernel32.def
 0001:00032f68       _PeekConsoleInputA@16      00043f68   kernel32:kernel32.def
 0001:00032f6e       _GetStdHandle@4            00043f6e   kernel32:kernel32.def
 0001:00032f74       _GetLocalTime@4            00043f74   kernel32:kernel32.def
 0001:00032f7a       _SetLocalTime@4            00043f7a   kernel32:kernel32.def
 0001:00032f80       _GetCurrentProcess@0       00043f80   kernel32:kernel32.def
 0001:00032f86       _SetFileAttributesA@8      00043f86   kernel32:kernel32.def
 0001:00032f8c       _SetHandleCount@4          00043f8c   kernel32:kernel32.def
 0001:00032f92       _SetErrorMode@4            00043f92   kernel32:kernel32.def
 0001:00032f98       _Sleep@4                   00043f98   kernel32:kernel32.def
 0001:00032f9e       _Beep@8                    00043f9e   kernel32:kernel32.def
 0001:00032fa4       _GetEnvironmentStrings@0   00043fa4   kernel32:kernel32.def
 0001:00032faa       _ExitProcess@4             00043faa   kernel32:kernel32.def
 0001:00032fb0       _GetLastError@0            00043fb0   kernel32:kernel32.def
 0001:00032fb6       _GetFileAttributesA@4      00043fb6   kernel32:kernel32.def
 0001:00032fbc       _SetFilePointer@16         00043fbc   kernel32:kernel32.def
 0001:00032fc2       _SetConsoleMode@8          00043fc2   kernel32:kernel32.def
 0001:00032fc8       _ReadConsoleInputA@16      00043fc8   kernel32:kernel32.def
 0001:00032fce       _GetConsoleMode@8          00043fce   kernel32:kernel32.def
 0001:00032fd4       _GetNumberOfConsoleInputEvents@8 00043fd4   kernel32:kernel32.def
 0001:00032fda       _WriteConsoleA@20          00043fda   kernel32:kernel32.def
 0001:00032fe0       _ReadConsoleA@20           00043fe0   kernel32:kernel32.def
 0001:00032fe6       _FindFirstFileA@8          00043fe6   kernel32:kernel32.def
 0001:00032fec       _FindNextFileA@8           00043fec   kernel32:kernel32.def
 0001:00032ff2       _FindClose@4               00043ff2   kernel32:kernel32.def
 0001:00032ff8       _FileTimeToSystemTime@8    00043ff8   kernel32:kernel32.def
 0001:00032ffe       _SetFileTime@16            00043ffe   kernel32:kernel32.def
 0001:00033004       _SystemTimeToFileTime@8    00044004   kernel32:kernel32.def
 0001:0003300a       _MoveFileA@8               0004400a   kernel32:kernel32.def
 0001:00033010       _DeleteFileA@4             00044010   kernel32:kernel32.def
 0001:00033016       _WriteFile@20              00044016   kernel32:kernel32.def
 0001:0003301c       _CloseHandle@4             0004401c   kernel32:kernel32.def
 0001:00033022       _GetFileType@4             00044022   kernel32:kernel32.def
 0001:00033028       _CreateFileA@28            00044028   kernel32:kernel32.def
 0001:0003302e       _WideCharToMultiByte@32    0004402e   kernel32:kernel32.def
 0001:00033034       _LCMapStringW@24           00044034   kernel32:kernel32.def
 0001:0003303a       _MultiByteToWideChar@24    0004403a   kernel32:kernel32.def
 0001:00033040       _SetEndOfFile@4            00044040   kernel32:kernel32.def
 0001:00033046       _SetEnvironmentVariableA@8 00044046   kernel32:kernel32.def
 0001:0003304c       _SetConsoleCtrlHandler@8   0004404c   kernel32:kernel32.def
 0001:00033052       _ReadFile@20               00044052   kernel32:kernel32.def
 0001:00033058       _RtlUnwind@16              00044058   kernel32:kernel32.def
 0001:0003305e       _UnhandledExceptionFilter@4 0004405e   kernel32:kernel32.def
 0001:00033064       _GetModuleFileNameA@12     00044064   kernel32:kernel32.def
 0001:0003306a       _GetStartupInfoA@4         0004406a   kernel32:kernel32.def
 0001:00033070       _VirtualFree@12            00044070   kernel32:kernel32.def
 0001:00033076       _VirtualAlloc@16           00044076   kernel32:kernel32.def
 0001:0003307c       _GetCurrentProcessId@0     0004407c   kernel32:kernel32.def
 0001:00033082       _SetStdHandle@8            00044082   kernel32:kernel32.def
 0001:00033088       _GetSystemTime@4           00044088   kernel32:kernel32.def
 0001:0003308e       _GetCurrentDirectoryA@8    0004408e   kernel32:kernel32.def
 0001:00033094       _GetFullPathNameA@16       00044094   kernel32:kernel32.def
 0001:0003309a       _GetLogicalDrives@0        0004409a   kernel32:kernel32.def
 0001:000330a0       _SetCurrentDirectoryA@4    000440a0   kernel32:kernel32.def
 0001:000330a6       _GetStringTypeW@16         000440a6   kernel32:kernel32.def
 0001:000330ac       _GetExitCodeProcess@8      000440ac   kernel32:kernel32.def
 0001:000330b2       _WaitForSingleObject@8     000440b2   kernel32:kernel32.def
 0001:000330b8       _CreateProcessA@40         000440b8   kernel32:kernel32.def
 0001:000330be       _RaiseException@16         000440be   kernel32:kernel32.def
 0001:000330c4       _FlushFileBuffers@4        000440c4   kernel32:kernel32.def
 0001:000330d0       __QWINGetDefaultWindow     000440d0 f console:console.obj
 0001:000330e5       __QWINGetFileName          000440e5 f console:console.obj
 0001:000330f7       __wgopen                   000440f7 f console:console.obj
 0001:00033109       __QWINClose                00044109 f console:console.obj
 0001:0003311b       __wgsetactive              0004411b f console:console.obj
 0001:0003312d       __wggetactive              0004412d f console:console.obj
 0001:0003313f       __QWINWrite                0004413f f console:console.obj
 0001:00033151       __QWINRead                 00044151 f console:console.obj
 0001:00033163       _YIELDQQ@0                 00044163 f console:console.obj
 0001:0003316e       __QWINSetSize              0004416e f console:console.obj
 0001:00033180       __QWINGetSize              00044180 f console:console.obj
 0001:00033192       __QWINMsgBox               00044192 f console:console.obj
 0001:000331a4       __QWINRegisterInit         000441a4 f console:console.obj
 0001:000331af       __QWINRegisterEnd          000441af f console:console.obj
 0001:000331ba       __QWINNiceExit             000441ba f console:console.obj
 0001:000331cc       __QWINSetFocus             000441cc f console:console.obj
 0002:00000000       _VDU                       00045000   <common>
 0002:00000018       _MOSPOS                    00045018   <common>
 0002:0000001c       _ARTEMIS                   0004501c   <common>
 0002:00000080       _AUX                       00045080   <common>
 0002:000000a8       _fpSetDescriptor           000450a8   <common>
 0002:000000ac       _fpGetDescriptor           000450ac   <common>
 0002:000000b0       _fpRealAlloc               000450b0   <common>
 0002:000000b4       _fpRealFree                000450b4   <common>
 0002:000000b8       _fpRealMap                 000450b8   <common>
 0002:000000bc       _fpRealCall                000450bc   <common>
 0002:000000c0       _fpRealIntr                000450c0   <common>
 0002:000000c4       _VideoSel                  000450c4   <common>
 0002:000000c8       _fpAllocDescriptor         000450c8   <common>
 0002:000000cc       __FFfirst                  000450cc   <common>
 0002:000000d0       __FFHack                   000450d0   <common>
 0002:000000d4       __matherr_flag             000450d4   <common>
 0002:000000d8       __aenvptr                  000450d8   <common>
 0002:000000dc       __bufin                    000450dc   <common>
 0002:000010dc       _matherr_flag              000460dc   <common>
 0002:000010e0       __heap_regions             000460e0   <common>
 0002:000013e0       __heap_descpages           000463e0   <common>
 0002:000013e4       __acmdln                   000463e4   <common>
 0002:000013e8       __pgmptr                   000463e8   <common>
 0002:000013ec       ___onexitend               000463ec   <common>
 0002:000013f0       ___onexitbegin             000463f0   <common>
 0002:00009bc0       _b$VesaStatus              0004ebc0   libf:llinit.obj
 0002:00009bc3       _b$VGAmodesH               0004ebc3   libf:llinit.obj
 0002:00009bc4       _b$WriteMode               0004ebc4   libf:llinit.obj
 0002:00009bc5       _b$EgaPalSup               0004ebc5   libf:llinit.obj
 0002:00009bc9       _b$CgaInfo                 0004ebc9   libf:llinit.obj
 0002:00009bca       _b$Adapter                 0004ebca   libf:llinit.obj
 0002:00009bcb       _b$Monitor                 0004ebcb   libf:llinit.obj
 0002:00009bcc       _b$VideoMem                0004ebcc   libf:llinit.obj
 0002:00009bd0       __qcg_status               0004ebd0   libf:qcinit.obj
 0002:00009bd1       _$_arc_info_fValid         0004ebd1   libf:qcinit.obj
 0002:00009be0       _VideoBaseTableLen         0004ebe0   libf:llcgrp.obj
 0002:00009be4       _b$MaskC                   0004ebe4   libf:llcgrp.obj
 0002:00009be4       _b$PenC                    0004ebe4   libf:llcgrp.obj
 0002:00009be5       _b$AttrC                   0004ebe5   libf:llcgrp.obj
 0002:00009be6       _b$AddrC                   0004ebe6   libf:llcgrp.obj
 0002:00009be6       _b$OffC                    0004ebe6   libf:llcgrp.obj
 0002:00009bea       _b$SegC                    0004ebea   libf:llcgrp.obj
 0002:00009bec       _b$PageC                   0004ebec   libf:llcgrp.obj
 0002:00009bee       _b$SaveCp                  0004ebee   libf:llcgrp.obj
 0002:00009bf0       _b$VesaWinFunc             0004ebf0   libf:llcgrp.obj
 0002:00009bf4       _b$PaintBorder             0004ebf4   libf:llcgrp.obj
 0002:00009bf5       _b$Tiling                  0004ebf5   libf:llcgrp.obj
 0002:00009bf6       _b$SaveCa                  0004ebf6   libf:llcgrp.obj
 0002:00009bfa       _b$SaveCm                  0004ebfa   libf:llcgrp.obj
 0002:00009bfb       _b$PlaneMask               0004ebfb   libf:llcgrp.obj
 0002:00009bfc       _b$Incr1                   0004ebfc   libf:llcgrp.obj
 0002:00009bfe       _b$Incr2                   0004ebfe   libf:llcgrp.obj
 0002:00009c00       _b$IncrY                   0004ec00   libf:llcgrp.obj
 0002:00009c02       _b$PageL                   0004ec02   libf:llcgrp.obj
 0002:00009c04       _B$VTOFST                  0004ec04   libf:llcgrp.obj
 0002:00009c0a       _B$VBOFST                  0004ec0a   libf:llcgrp.obj
 0002:00009c10       _B$LEOFST                  0004ec10   libf:llcgrp.obj
 0002:00009c16       _B$REOFST                  0004ec16   libf:llcgrp.obj
 0002:00009c1c       _B$VLOFST                  0004ec1c   libf:llcgrp.obj
 0002:00009c20       _B$VROFST                  0004ec20   libf:llcgrp.obj
 0002:00009c24       _B$VLMASK                  0004ec24   libf:llcgrp.obj
 0002:00009c25       _B$VRMASK                  0004ec25   libf:llcgrp.obj
 0002:00009c26       _b$BorderColor             0004ec26   libf:llcgrp.obj
 0002:00009c50       _$_current_x               0004ec50   libf:qcdata.obj
 0002:00009c52       _$_current_y               0004ec52   libf:qcdata.obj
 0002:00009c54       _$_bkg_color               0004ec54   libf:qcdata.obj
 0002:00009c58       _$_txt_fg_color            0004ec58   libf:qcdata.obj
 0002:00009c59       _$_text_attrib             0004ec59   libf:qcdata.obj
 0002:00009c5a       _$_line_style_mask         0004ec5a   libf:qcdata.obj
 0002:00009c5c       _$_fill_mask               0004ec5c   libf:qcdata.obj
 0002:00009c64       _$_fill_mask_p             0004ec64   libf:qcdata.obj
 0002:00009c65       _$_BKG_MASK                0004ec65   libf:qcdata.obj
 0002:00009c75       _$LINE_DRAWN               0004ec75   libf:qcdata.obj
 0002:00009c77       _$_text_row                0004ec77   libf:qcdata.obj
 0002:00009c79       _$_text_column             0004ec79   libf:qcdata.obj
 0002:00009c7b       _$_text_org_row            0004ec7b   libf:qcdata.obj
 0002:00009c7d       _$_text_org_col            0004ec7d   libf:qcdata.obj
 0002:00009c7f       _$_text_max_row            0004ec7f   libf:qcdata.obj
 0002:00009c81       _$_text_max_col            0004ec81   libf:qcdata.obj
 0002:00009c83       _$_off_screen              0004ec83   libf:qcdata.obj
 0002:00009c84       _$_text_wrap_p             0004ec84   libf:qcdata.obj
 0002:00009c85       _$_cursor_on_screen        0004ec85   libf:qcdata.obj
 0002:00009c86       _$_old_mode                0004ec86   libf:qcdata.obj
 0002:00009c88       _b$Buf1                    0004ec88   libf:qcdata.obj
 0002:00009d22       _B$VesaModeInfo            0004ed22   libf:llvesa.obj
 0002:00009d62       _b$VesaWin                 0004ed62   libf:llvesa.obj
 0002:00009d64       _b$FastVesa                0004ed64   libf:llvesa.obj
 0002:00009d92       _regs16                    0004ed92   libf:llvesa.obj
 0002:00009dae       _retVal                    0004edae   libf:llvesa.obj
 0002:00009db2       _b$VesaRealSeg             0004edb2   libf:llvesa.obj
 0002:00009db4       _b$WinFuncPtr              0004edb4   libf:llvesa.obj
 0002:00009dd0       _B$GRPACX                  0004edd0   libf:grdata.obj
 0002:00009dd2       _B$GRPACY                  0004edd2   libf:grdata.obj
 0002:00009dd4       _B$GX_OLD                  0004edd4   libf:grdata.obj
 0002:00009dd8       _B$GY_OLD                  0004edd8   libf:grdata.obj
 0002:00009ddc       _B$GXPOS                   0004eddc   libf:grdata.obj
 0002:00009dde       _B$GYPOS                   0004edde   libf:grdata.obj
 0002:00009de0       _B$GRFACX                  0004ede0   libf:grdata.obj
 0002:00009de4       _B$GRFACY                  0004ede4   libf:grdata.obj
 0002:00009de8       _B$LINSTL                  0004ede8   libf:grdata.obj
 0002:00009dea       _B$CLINEF                  0004edea   libf:grdata.obj
 0002:00009deb       _b$ASPECTR                 0004edeb   libf:grdata.obj
 0002:00009ded       _B$CENCNT                  0004eded   libf:grdata.obj
 0002:00009def       _B$CNPNTS                  0004edef   libf:grdata.obj
 0002:00009df1       _B$CSTCNT                  0004edf1   libf:grdata.obj
 0002:00009df3       _B$CPLOTF                  0004edf3   libf:grdata.obj
 0002:00009df4       _B$COPTFL                  0004edf4   libf:grdata.obj
 0002:00009df5       _B$TILLOC                  0004edf5   libf:grdata.obj
 0002:00009df9       _B$TILFLG                  0004edf9   libf:grdata.obj
 0002:00009dfa       _B$TILNDX                  0004edfa   libf:grdata.obj
 0002:00009dfb       _B$TILLEN                  0004edfb   libf:grdata.obj
 0002:00009dfc       _B$TILHGT                  0004edfc   libf:grdata.obj
 0002:00009dfd       _B$TILPTR                  0004edfd   libf:grdata.obj
 0002:00009dfe       _B$GRPLAN                  0004edfe   libf:grdata.obj
 0002:00009dff       _B$WNDWSW                  0004edff   libf:grdata.obj
 0002:00009e00       _B$WNDWSC                  0004ee00   libf:grdata.obj
 0002:00009e01       _B$VIEWSW                  0004ee01   libf:grdata.obj
 0002:00009e10       _b$EgaPalette              0004ee10   libf:llxgasup.obj
 0002:00009e40       _B$VXSIZ                   0004ee40   libf:grinit.obj
 0002:00009e42       _B$VYSIZ                   0004ee42   libf:grinit.obj
 0002:00009e44       _B$VXMIN                   0004ee44   libf:grinit.obj
 0002:00009e46       _B$VXMAX                   0004ee46   libf:grinit.obj
 0002:00009e48       _B$VYMIN                   0004ee48   libf:grinit.obj
 0002:00009e4a       _B$VYMAX                   0004ee4a   libf:grinit.obj
 0002:00009e4c       _B$VXOFF                   0004ee4c   libf:grinit.obj
 0002:00009e4e       _B$VYOFF                   0004ee4e   libf:grinit.obj
 0002:00009e50       _B$VXDIF                   0004ee50   libf:grinit.obj
 0002:00009e52       _B$VYDIF                   0004ee52   libf:grinit.obj
 0002:00009e60       ___FCclenv                 0004ee60   libf:qcdumb.obj
 0002:00009e62       ___asizeC                  0004ee62   libf:qcdumb.obj
 0002:00009e63       ___osmode                  0004ee63   libf:qcdumb.obj
 0002:00009e64       ___osmajor                 0004ee64   libf:qcdumb.obj
 0002:00009e70       _b$PageTable               0004ee70   libf:lltext.obj
 0002:00009ee0       _b$UpSub                   0004eee0   libf:llcgasup.obj
 0002:00009ee2       _b$DnSub                   0004eee2   libf:llcgasup.obj
 0002:00009ee4       _b$UpDnAdd                 0004eee4   libf:llcgasup.obj
 0002:00009ef0       _b$IncrYHi                 0004eef0   libf:llegasup.obj
 0002:00009f20       _B$PXDIF                   0004ef20   libf:qcfpvars.obj
 0002:00009f28       _B$PYDIF                   0004ef28   libf:qcfpvars.obj
 0002:00009f30       _B$LXDIF                   0004ef30   libf:qcfpvars.obj
 0002:00009f38       _B$LYDIF                   0004ef38   libf:qcfpvars.obj
 0002:00009f40       _B$WXMIN                   0004ef40   libf:qcfpvars.obj
 0002:00009f48       _B$WYMIN                   0004ef48   libf:qcfpvars.obj
 0002:00009f50       _B$WXMAX                   0004ef50   libf:qcfpvars.obj
 0002:00009f58       _B$WYMAX                   0004ef58   libf:qcfpvars.obj
 0002:00009f60       _$_wxycoord                0004ef60   libf:qcfpsup.obj
 0002:00009f70       _b$ScratchW                0004ef70   libf:grwindow.obj
 0003:00000268       __FFherrout                00050268   libf:core.obj
 0003:00000270       __FFldintfmt               00050270   libf:core.obj
 0003:00000288       __FFmaxunits               00050288   libf:unit.obj
 0004:000054f8       __FFopAccess_tab           000564f8   libf:opn.obj
 0004:00005518       __FFopBlank_tab            00056518   libf:opn.obj
 0004:00005528       __FFopStatus_tab           00056528   libf:opn.obj
 0004:00005548       __FFopForm_tab             00056548   libf:opn.obj
 0004:00005570       __FFopShare_tab            00056570   libf:opn.obj
 0004:000055a0       __FFopMode_tab             000565a0   libf:opn.obj
 0004:000055c0       __FFtable_tab              000565c0   libf:opn.obj
 0004:000055e8       __FFtypetable              000565e8   libf:opn.obj
 0004:00005600       _inqMode_tab               00056600   libf:inq.obj
 0004:00005604       _inqShare_tab              00056604   libf:inq.obj
 0004:00005610       _inqAccess_tab             00056610   libf:inq.obj
 0004:00005618       _inqForm_tab               00056618   libf:inq.obj
 0004:000056c0       _inq_s_table               000566c0   libf:inq.obj
 0004:00005760       __FFclStatus_tab           00056760   libf:cls.obj
 0004:000057a4       __FFpharlap                000567a4   libf:fortstr.obj
 0004:00005808       __FFzero                   00056808   libf:intrin.obj
 0004:00005810       __FFhalf                   00056810   libf:intrin.obj
 0004:00005818       __FFone                    00056818   libf:intrin.obj
 0004:00005820       __FFtwo                    00056820   libf:intrin.obj
 0004:00005828       __FFten                    00056828   libf:intrin.obj
 0004:00005830       __FFline                   00056830   libf:intrin.obj
 0004:000058e8       _blanks                    000568e8   libf:tab.obj
 0004:00005ae0       ___QCGdummy                00056ae0   libf:fginit.obj
 0004:00005af0       _b$UsrCsrTyp               00056af0   libf:llinit.obj
 0004:00005af2       _b$OrgCsrTyp               00056af2   libf:llinit.obj
 0004:00005af4       _b$OrgBiosMode             00056af4   libf:llinit.obj
 0004:00005af7       _b$orglen                  00056af7   libf:llinit.obj
 0004:00005b00       _b$ScreenX                 00056b00   libf:qcinit.obj
 0004:00005b61       _$_new_height              00056b61   libf:qcinit.obj
 0004:00005b62       _MyMaxBiosMode             00056b62   libf:qcinit.obj
 0004:00005b70       _b$ModeData                00056b70   libf:llcgrp.obj
 0004:00005b70       _b$ScreenMode              00056b70   libf:llcgrp.obj
 0004:00005b71       _b$Burst                   00056b71   libf:llcgrp.obj
 0004:00005b72       _b$BiosMode                00056b72   libf:llcgrp.obj
 0004:00005b74       _b$ScrWidth                00056b74   libf:llcgrp.obj
 0004:00005b75       _b$ScrHeight               00056b75   libf:llcgrp.obj
 0004:00005b76       _b$HorzRes                 00056b76   libf:llcgrp.obj
 0004:00005b78       _b$VertRes                 00056b78   libf:llcgrp.obj
 0004:00005b7a       _b$VideoBase               00056b7a   libf:llcgrp.obj
 0004:00005b7c       _b$MaxAttr                 00056b7c   libf:llcgrp.obj
 0004:00005b7d       _b$MaxColor                00056b7d   libf:llcgrp.obj
 0004:00005b7e       _b$PageSize                00056b7e   libf:llcgrp.obj
 0004:00005b7f       _b$CurrPSize               00056b7f   libf:llcgrp.obj
 0004:00005b81       _b$MaxPage                 00056b81   libf:llcgrp.obj
 0004:00005b82       _b$FBColors                00056b82   libf:llcgrp.obj
 0004:00005b82       _b$ForeColor               00056b82   libf:llcgrp.obj
 0004:00005b83       _b$EgaWrMd                 00056b83   libf:llcgrp.obj
 0004:00005b84       _b$InitPalette             00056b84   libf:llcgrp.obj
 0004:00005b88       _b$InitVgaPal              00056b88   libf:llcgrp.obj
 0004:00005b8c       _b$SetMode                 00056b8c   libf:llcgrp.obj
 0004:00005b90       _b$SetPages                00056b90   libf:llcgrp.obj
 0004:00005b94       _b$PalReset                00056b94   libf:llcgrp.obj
 0004:00005b98       _b$PalPut                  00056b98   libf:llcgrp.obj
 0004:00005b9c       _b$PalTrans                00056b9c   libf:llcgrp.obj
 0004:00005ba0       _b$PalSet                  00056ba0   libf:llcgrp.obj
 0004:00005ba4       _b$BitsPerPixel            00056ba4   libf:llcgrp.obj
 0004:00005ba5       _b$Planes                  00056ba5   libf:llcgrp.obj
 0004:00005ba6       _b$BytesPerRow             00056ba6   libf:llcgrp.obj
 0004:00005ba8       _b$MaskLeft                00056ba8   libf:llcgrp.obj
 0004:00005ba9       _b$MaskRight               00056ba9   libf:llcgrp.obj
 0004:00005baa       _b$PixelsPerByte           00056baa   libf:llcgrp.obj
 0004:00005bac       _b$DivShift                00056bac   libf:llcgrp.obj
 0004:00005bad       _b$ModMask                 00056bad   libf:llcgrp.obj
 0004:00005baf       _b$Aspect                  00056baf   libf:llcgrp.obj
 0004:00005bb1       _b$AspectInv               00056bb1   libf:llcgrp.obj
 0004:00005bb3       _b$MapXYC                  00056bb3   libf:llcgrp.obj
 0004:00005bb7       _b$LeftC                   00056bb7   libf:llcgrp.obj
 0004:00005bbb       _b$ChkUpC                  00056bbb   libf:llcgrp.obj
 0004:00005bbf       _b$UpC                     00056bbf   libf:llcgrp.obj
 0004:00005bc3       _b$ChkDownC                00056bc3   libf:llcgrp.obj
 0004:00005bc7       _b$DownC                   00056bc7   libf:llcgrp.obj
 0004:00005bcb       _b$SetAttr                 00056bcb   libf:llcgrp.obj
 0004:00005bcf       _b$ReadC                   00056bcf   libf:llcgrp.obj
 0004:00005bd3       _b$SetC                    00056bd3   libf:llcgrp.obj
 0004:00005bd7       _b$SetPixC                 00056bd7   libf:llcgrp.obj
 0004:00005bdb       _b$SetPixFirstC            00056bdb   libf:llcgrp.obj
 0004:00005bdf       _b$SetPixLastC             00056bdf   libf:llcgrp.obj
 0004:00005be3       _b$LineX                   00056be3   libf:llcgrp.obj
 0004:00005be7       _b$LineY                   00056be7   libf:llcgrp.obj
 0004:00005beb       _b$LineV                   00056beb   libf:llcgrp.obj
 0004:00005bef       _b$PutAction               00056bef   libf:llcgrp.obj
 0004:00005bf3       _b$NReadL                  00056bf3   libf:llcgrp.obj
 0004:00005bf7       _b$NWriteL                 00056bf7   libf:llcgrp.obj
 0004:00005bfb       _b$NSetC                   00056bfb   libf:llcgrp.obj
 0004:00005bff       _b$PaintBound              00056bff   libf:llcgrp.obj
 0004:00005c03       _b$SetTile                 00056c03   libf:llcgrp.obj
 0004:00005c07       _b$ScanL                   00056c07   libf:llcgrp.obj
 0004:00005c0b       _b$ScanR                   00056c0b   libf:llcgrp.obj
 0004:00005c0f       _b$PutVector               00056c0f   libf:llcgrp.obj
 0004:00005d80       __FFstktop                 00056d80   libf:core.obj
 0004:00005d84       __FFstkbot                 00056d84   libf:core.obj
 0004:00005d88       __FFstksize                00056d88   libf:core.obj
 0004:00005d90       __FFgd                     00056d90   libf:core.obj
 0004:00005ff0       __FFTerminate              00056ff0   libf:core.obj
 0004:00005ff4       __FFconfig                 00056ff4   libf:core.obj
 0004:00005ff8       __FFfn                     00056ff8   libf:core.obj
 0004:00006100       __FFtype                   00057100   libf:core.obj
 0004:00006110       __FFdatasizes              00057110   libf:core.obj
 0004:00006140       __FFldfltfmt               00057140   libf:core.obj
 0004:00006170       __FFffsequence             00057170   libf:core.obj
 0004:00006178       __FFnewline                00057178   libf:core.obj
 0004:000061c8       __pFFinit                  000571c8   libf:core.obj
 0004:000061d0       __FFshare_tab              000571d0   libf:core.obj
 0004:000061d8       __FFmode_tab               000571d8   libf:core.obj
 0004:000061e0       __FFdevice_info            000571e0   libf:core.obj
 0004:00006228       __FFdefault_tab            00057228   libf:core.obj
 0004:00006448       __FFunit_lst               00057448   libf:unit.obj
 0004:00006678       __FFnextreci_handlers      00057678   libf:iodec2.obj
 0004:00006688       __FFnextreco_handlers      00057688   libf:iodec2.obj
 0004:00006698       __FFoutput_processors      00057698   libf:iodec2.obj
 0004:000066a4       __FFinput_processors       000576a4   libf:iodec2.obj
 0004:000066b0       __FFnum_fetchers           000576b0   libf:iodec2.obj
 0004:000066b8       __FFchn_fetchers           000576b8   libf:iodec2.obj
 0004:000066c0       __FFbyte_senders           000576c0   libf:iodec2.obj
 0004:000066c8       __FFunf_rtn_tab            000576c8   libf:iodec2.obj
 0004:000066e0       __FFflt_decoder            000576e0   libf:iodec2.obj
 0004:000066e4       __FFflt_encoder            000576e4   libf:iodec2.obj
 0004:000066e8       __FFhex_handler            000576e8   libf:iodec2.obj
 0004:000066f8       __FFdummy                  000576f8   libf:finit.obj
 0004:00006700       _ulMaxVals                 00057700   libf:fstrtol.obj
 0004:00006790       __FFexcept                 00057790   libf:matherr.obj
 0004:00006960       _b$SavedWin                00057960   libf:qccore.obj
 0004:00006970       _scanlinebytes             00057970   libf:qccore.obj
 0004:00006980       _$_cursor_enabled          00057980   libf:qcdata.obj
 0004:00006981       _B$SEG_ZERO                00057981   libf:qcdata.obj
 0004:00006983       _B$SEG_MDPA                00057983   libf:qcdata.obj
 0004:00006985       _B$SEG_CGA                 00057985   libf:qcdata.obj
 0004:00006987       _B$SEG_EGA                 00057987   libf:qcdata.obj
 0004:00006989       _B$SEG_VGA                 00057989   libf:qcdata.obj
 0004:0000698b       _B$SEG_MCGA                0005798b   libf:qcdata.obj
 0004:0000698d       _B$SEG_HGC                 0005798d   libf:qcdata.obj
 0004:0000698f       _B$SEG_OGA                 0005798f   libf:qcdata.obj
 0004:00006991       _B$SEG_VESA                00057991   libf:qcdata.obj
 0004:00006993       _B$SEG_SuperVGA            00057993   libf:qcdata.obj
 0004:00006995       _B$SEG_FUNCTABLE           00057995   libf:qcdata.obj
 0004:00006997       _B$SEG_OLI_SYS             00057997   libf:qcdata.obj
 0004:00006999       _B$SEG_OLI_ROM             00057999   libf:qcdata.obj
 0004:0000699b       _B$SEG_OLI_OPTIONS         0005799b   libf:qcdata.obj
 0004:0000699d       _b$BlockSel                0005799d   libf:qcdata.obj
 0004:0000699f       _b$BlockRealSeg            0005799f   libf:qcdata.obj
 0004:000069a1       _b$prev1FVector            000579a1   libf:qcdata.obj
 0004:000069a5       _b$VideoBaseTable          000579a5   libf:qcdata.obj
 0004:000069ab       _b$SelectorTable           000579ab   libf:qcdata.obj
 0004:000069bd       _b$EGASelTable             000579bd   libf:qcdata.obj
 0004:000069cf       _b$EGAPagAddrs             000579cf   libf:qcdata.obj
 0004:000069e0       _b$CSRTYP                  000579e0   libf:llcscn.obj
 0004:000069e2       _b$CurPages                000579e2   libf:llcscn.obj
 0004:000069e2       _b$ActPage                 000579e2   libf:llcscn.obj
 0004:000069e3       _b$VisPage                 000579e3   libf:llcscn.obj
 0004:00006a12       _b$VgaPalette              00057a12   libf:llvga.obj
 0004:00006dc0       __GTextVect                00057dc0   libf:fontchar.obj
 0004:00006ee0       ____aDBswpflg              00057ee0   libf:qcdumb.obj
 0004:00006ee2       ____aDBswpchk              00057ee2   libf:qcdumb.obj
 0004:00006f38       __FFerrnum                 00057f38   libf:build.obj
 0004:00006f40       __FFermsg                  00057f40   libf:build.obj
 0004:00006f58       __FFDefMathErr             00057f58   libf:mhandler.obj
 0004:00006f60       _b$Mode2Palette            00057f60   libf:llcgasup.obj
 0004:00006f62       _b$Mode2VgaPal             00057f62   libf:llcgasup.obj
 0004:00006fd8       __FFerrors                 00057fd8   libf:errdic.obj
 0004:00006fe0       __FFer_index               00057fe0   libf:errdic.obj
 0004:00007420       __FFer_buffer              00058420   libf:errdic.obj
 0004:00007920       __FFtmap                   00058920   libf:errmap.obj
 0004:00007ae4       __aexit_rtn                00058ae4   libc:CRT0.OBJ
 0004:00007ae8       __fltused                  00058ae8   libc:fpinit.obj
 0004:00007aec       __ldused                   00058aec   libc:fpinit.obj
 0004:00007af0       ___fastflag                00058af0   libc:fpinit.obj
 0004:00007af4       __FPinit                   00058af4   libc:fpinit.obj
 0004:00007af8       __FPmtinit                 00058af8   libc:fpinit.obj
 0004:00007afc       __FPmtterm                 00058afc   libc:fpinit.obj
 0004:00007b00       __pnhHeap                  00058b00   libc:MALLOC.OBJ
 0004:00007b04       _errno                     00058b04   libc:CRT0DAT.OBJ
 0004:00007b08       __doserrno                 00058b08   libc:CRT0DAT.OBJ
 0004:00007b0c       __umaskval                 00058b0c   libc:CRT0DAT.OBJ
 0004:00007b10       __osver                    00058b10   libc:CRT0DAT.OBJ
 0004:00007b14       __winver                   00058b14   libc:CRT0DAT.OBJ
 0004:00007b18       __winmajor                 00058b18   libc:CRT0DAT.OBJ
 0004:00007b1c       __winminor                 00058b1c   libc:CRT0DAT.OBJ
 0004:00007b20       ___argc                    00058b20   libc:CRT0DAT.OBJ
 0004:00007b24       ___argv                    00058b24   libc:CRT0DAT.OBJ
 0004:00007b28       __environ                  00058b28   libc:CRT0DAT.OBJ
 0004:00007b2c       __exitflag                 00058b2c   libc:CRT0DAT.OBJ
 0004:00007b30       __C_Termination_Done       00058b30   libc:CRT0DAT.OBJ
 0004:00007b58       __OP_FMODjmptab            00058b58   libc:87fmod.obj
 0004:00007ba8       __timezone                 00058ba8   libc:TIMESET.OBJ
 0004:00007bac       __daylight                 00058bac   libc:TIMESET.OBJ
 0004:00007bb8       __tzname                   00058bb8   libc:TIMESET.OBJ
 0004:00007bc0       ___dnames                  00058bc0   libc:TIMESET.OBJ
 0004:00007bd8       ___mnames                  00058bd8   libc:TIMESET.OBJ
 0004:000081b8       __adbgmsg                  000591b8   libc:CRT0MSG.OBJ
 0004:000081d0       __XcptActTab               000591d0   libc:WINXFLTR.OBJ
 0004:00008248       __XcptActTabCount          00059248   libc:WINXFLTR.OBJ
 0004:0000824c       __fpecode                  0005924c   libc:WINXFLTR.OBJ
 0004:00008250       __pxcptinfoptrs            00059250   libc:WINXFLTR.OBJ
 0004:00008258       __nhandle                  00059258   libc:IOINIT.OBJ
 0004:00008260       __osfile                   00059260   libc:IOINIT.OBJ
 0004:000082a0       __osfhnd                   000592a0   libc:IOINIT.OBJ
 0004:000083a0       __pipech                   000593a0   libc:IOINIT.OBJ
 0004:000083e0       __heap_desc                000593e0   libc:HEAPINIT.OBJ
 0004:000083f4       __heap_resetsize           000593f4   libc:HEAPINIT.OBJ
 0004:000083f8       __amblksiz                 000593f8   libc:HEAPINIT.OBJ
 0004:000083fc       __heap_regionsize          000593fc   libc:HEAPINIT.OBJ
 0004:00008400       __heap_maxregsize          00059400   libc:HEAPINIT.OBJ
 0004:00008408       __cfltcvt_tab              00059408   libc:CMISCDAT.OBJ
 0004:00008526       __OP_SINjmptab             00059526   libc:87trig.obj
 0004:00008546       __OP_COSjmptab             00059546   libc:87trig.obj
 0004:00008566       __OP_TANjmptab             00059566   libc:87trig.obj
 0004:00008588       __OP_SINHjmptab            00059588   libc:87trigh.obj
 0004:000085a8       __OP_COSHjmptab            000595a8   libc:87trigh.obj
 0004:000085c8       __OP_TANHjmptab            000595c8   libc:87trigh.obj
 0004:000085e8       __infinity                 000595e8   libc:87tran.obj
 0004:000085f2       __minfinity                000595f2   libc:87tran.obj
 0004:000085fc       __logemax                  000595fc   libc:87tran.obj
 0004:0000862c       __OP_POWjmptab             0005962c   libc:87tran.obj
 0004:0000867c       __OP_LOG10jmptab           0005967c   libc:87tran.obj
 0004:0000869c       __OP_LOGjmptab             0005969c   libc:87tran.obj
 0004:000086bc       __OP_EXPjmptab             000596bc   libc:87tran.obj
 0004:000086dc       __OP_ASINjmptab            000596dc   libc:87triga.obj
 0004:000086fc       __OP_ACOSjmptab            000596fc   libc:87triga.obj
 0004:0000871c       __OP_ATANjmptab            0005971c   libc:87triga.obj
 0004:0000873c       __OP_ATAN2jmptab           0005973c   libc:87triga.obj
 0004:0000878c       __OP_SQRTjmptab            0005978c   libc:87sqrt.obj
 0004:000087ac       __indefinite               000597ac   libc:87disp.obj
 0004:000087b6       __piby2                    000597b6   libc:87disp.obj
 0004:000087c8       __cpower                   000597c8   libc:87disp.obj
 0004:000087e0       __lpdays                   000597e0   libc:DAYS.OBJ
 0004:00008818       __days                     00059818   libc:DAYS.OBJ
 0004:0000884c       __coninpfh                 0005984c   libc:CINITCON.OBJ
 0004:00008850       __confh                    00059850   libc:CINITCON.OBJ
 0004:0000887c       ___c_onexit                0005987c   libc:CINITONE.OBJ
 0004:00008880       __pctype                   00059880   libc:CTYPE.OBJ
 0004:00008884       __pwctype                  00059884   libc:CTYPE.OBJ
 0004:00008888       __ctype                    00059888   libc:CTYPE.OBJ
 0004:00008a8c       ___mb_cur_max              00059a8c   libc:NLSDATA1.OBJ
 0004:00008a94       __decimal_point            00059a94   libc:NLSDATA1.OBJ
 0004:00008a98       __decimal_point_length     00059a98   libc:NLSDATA1.OBJ
 0004:00008a9c       __fmode                    00059a9c   libc:TXTMODE.OBJ
 0004:00008aa0       __lc_handle                00059aa0   libc:NLSDATA2.OBJ
 0004:00008ab8       __lc_codepage              00059ab8   libc:NLSDATA2.OBJ
 0004:00008ac0       __stdbuf                   00059ac0   libc:_SFTBUF.OBJ
 0004:00008ac8       __iob                      00059ac8   libc:_FILE.OBJ
 0004:00008d48       __lastiob                  00059d48   libc:_FILE.OBJ
 0004:00008d4c       __p_overlay                00059d4c   libc:DOSPAWN.OBJ
 0004:00008d60       __cflush                   00059d60   libc:CINITSTD.OBJ
 0004:00008d68       __pow10pos                 00059d68   libc:constpow.obj
 0004:00008ec8       __pow10neg                 00059ec8   libc:constpow.obj
 0004:000091d8       __d_inf                    0005a1d8   libc:util.obj
 0004:000091e0       __d_ind                    0005a1e0   libc:util.obj
 0004:000091e8       __d_max                    0005a1e8   libc:util.obj
 0004:000091f0       __d_min                    0005a1f0   libc:util.obj
 0004:000091f8       __d_mzero                  0005a1f8   libc:util.obj
 0004:00009200       __qw32used                 0005a200   console:console.obj
 0004:00009208       ___xc_a                    0005a208   libc:crt0init.obj
 0004:00009210       ___xc_z                    0005a210   libc:crt0init.obj
 0004:00009218       ___xi_a                    0005a218   libc:crt0init.obj
 0004:00009248       ___xi_z                    0005a248   libc:crt0init.obj
 0004:00009250       ___xp_a                    0005a250   libc:crt0init.obj
 0004:00009260       ___xp_z                    0005a260   libc:crt0init.obj
 0004:00009268       ___xt_a                    0005a268   libc:crt0init.obj
 0004:00009270       ___xt_z                    0005a270   libc:crt0init.obj
 0005:00000000       _b$FP_1                    0005b000   libf:grdata.obj
 0005:00000004       _b$FP_256                  0005b004   libf:grdata.obj
 0005:00000008       _B$VIEWSC                  0005b008   libf:grdata.obj
 0006:00000000       KERNEL32_IMPORT_DESCRIPTOR 0005c000   kernel32:kernel32.def
 0006:00000014       NULL_IMPORT_DESCRIPTOR     0005c014   kernel32:kernel32.def
 0006:00000128       __imp__DeleteFileA@4       0005c128   kernel32:kernel32.def
 0006:0000012c       __imp__GetVersion@0        0005c12c   kernel32:kernel32.def
 0006:00000130       __imp__GetProcAddress@8    0005c130   kernel32:kernel32.def
 0006:00000134       __imp__LoadLibraryA@4      0005c134   kernel32:kernel32.def
 0006:00000138       __imp__PeekConsoleInputA@16 0005c138   kernel32:kernel32.def
 0006:0000013c       __imp__GetStdHandle@4      0005c13c   kernel32:kernel32.def
 0006:00000140       __imp__GetLocalTime@4      0005c140   kernel32:kernel32.def
 0006:00000144       __imp__SetLocalTime@4      0005c144   kernel32:kernel32.def
 0006:00000148       __imp__GetCurrentProcess@0 0005c148   kernel32:kernel32.def
 0006:0000014c       __imp__SetFileAttributesA@8 0005c14c   kernel32:kernel32.def
 0006:00000150       __imp__SetHandleCount@4    0005c150   kernel32:kernel32.def
 0006:00000154       __imp__SetErrorMode@4      0005c154   kernel32:kernel32.def
 0006:00000158       __imp__Sleep@4             0005c158   kernel32:kernel32.def
 0006:0000015c       __imp__Beep@8              0005c15c   kernel32:kernel32.def
 0006:00000160       __imp__GetEnvironmentStrings@0 0005c160   kernel32:kernel32.def
 0006:00000164       __imp__ExitProcess@4       0005c164   kernel32:kernel32.def
 0006:00000168       __imp__GetLastError@0      0005c168   kernel32:kernel32.def
 0006:0000016c       __imp__GetFileAttributesA@4 0005c16c   kernel32:kernel32.def
 0006:00000170       __imp__SetFilePointer@16   0005c170   kernel32:kernel32.def
 0006:00000174       __imp__SetConsoleMode@8    0005c174   kernel32:kernel32.def
 0006:00000178       __imp__ReadConsoleInputA@16 0005c178   kernel32:kernel32.def
 0006:0000017c       __imp__GetConsoleMode@8    0005c17c   kernel32:kernel32.def
 0006:00000180       __imp__GetNumberOfConsoleInputEvents@8 0005c180   kernel32:kernel32.def
 0006:00000184       __imp__WriteConsoleA@20    0005c184   kernel32:kernel32.def
 0006:00000188       __imp__ReadConsoleA@20     0005c188   kernel32:kernel32.def
 0006:0000018c       __imp__FindFirstFileA@8    0005c18c   kernel32:kernel32.def
 0006:00000190       __imp__FindNextFileA@8     0005c190   kernel32:kernel32.def
 0006:00000194       __imp__FindClose@4         0005c194   kernel32:kernel32.def
 0006:00000198       __imp__FileTimeToSystemTime@8 0005c198   kernel32:kernel32.def
 0006:0000019c       __imp__SetFileTime@16      0005c19c   kernel32:kernel32.def
 0006:000001a0       __imp__SystemTimeToFileTime@8 0005c1a0   kernel32:kernel32.def
 0006:000001a4       __imp__MoveFileA@8         0005c1a4   kernel32:kernel32.def
 0006:000001a8       __imp__GetCommandLineA@0   0005c1a8   kernel32:kernel32.def
 0006:000001ac       __imp__WriteFile@20        0005c1ac   kernel32:kernel32.def
 0006:000001b0       __imp__CloseHandle@4       0005c1b0   kernel32:kernel32.def
 0006:000001b4       __imp__GetFileType@4       0005c1b4   kernel32:kernel32.def
 0006:000001b8       __imp__CreateFileA@28      0005c1b8   kernel32:kernel32.def
 0006:000001bc       __imp__WideCharToMultiByte@32 0005c1bc   kernel32:kernel32.def
 0006:000001c0       __imp__LCMapStringW@24     0005c1c0   kernel32:kernel32.def
 0006:000001c4       __imp__MultiByteToWideChar@24 0005c1c4   kernel32:kernel32.def
 0006:000001c8       __imp__SetEndOfFile@4      0005c1c8   kernel32:kernel32.def
 0006:000001cc       __imp__SetEnvironmentVariableA@8 0005c1cc   kernel32:kernel32.def
 0006:000001d0       __imp__SetConsoleCtrlHandler@8 0005c1d0   kernel32:kernel32.def
 0006:000001d4       __imp__ReadFile@20         0005c1d4   kernel32:kernel32.def
 0006:000001d8       __imp__RtlUnwind@16        0005c1d8   kernel32:kernel32.def
 0006:000001dc       __imp__UnhandledExceptionFilter@4 0005c1dc   kernel32:kernel32.def
 0006:000001e0       __imp__GetModuleFileNameA@12 0005c1e0   kernel32:kernel32.def
 0006:000001e4       __imp__GetStartupInfoA@4   0005c1e4   kernel32:kernel32.def
 0006:000001e8       __imp__VirtualFree@12      0005c1e8   kernel32:kernel32.def
 0006:000001ec       __imp__VirtualAlloc@16     0005c1ec   kernel32:kernel32.def
 0006:000001f0       __imp__GetCurrentProcessId@0 0005c1f0   kernel32:kernel32.def
 0006:000001f4       __imp__SetStdHandle@8      0005c1f4   kernel32:kernel32.def
 0006:000001f8       __imp__GetSystemTime@4     0005c1f8   kernel32:kernel32.def
 0006:000001fc       __imp__GetCurrentDirectoryA@8 0005c1fc   kernel32:kernel32.def
 0006:00000200       __imp__GetFullPathNameA@16 0005c200   kernel32:kernel32.def
 0006:00000204       __imp__GetLogicalDrives@0  0005c204   kernel32:kernel32.def
 0006:00000208       __imp__SetCurrentDirectoryA@4 0005c208   kernel32:kernel32.def
 0006:0000020c       __imp__GetStringTypeW@16   0005c20c   kernel32:kernel32.def
 0006:00000210       __imp__GetExitCodeProcess@8 0005c210   kernel32:kernel32.def
 0006:00000214       __imp__WaitForSingleObject@8 0005c214   kernel32:kernel32.def
 0006:00000218       __imp__CreateProcessA@40   0005c218   kernel32:kernel32.def
 0006:0000021c       __imp__RaiseException@16   0005c21c   kernel32:kernel32.def
 0006:00000220       __imp__FlushFileBuffers@4  0005c220   kernel32:kernel32.def
 0006:00000224       \177KERNEL32__imp__NULL    0005c224   kernel32:kernel32.def

 entry point at        0001:00028d70

 Static symbols

 0001:000236e0       __PointFont                000346e0 f libf:fontlib.obj
 0001:00023708       __EnumFont                 00034708 f libf:fontlib.obj
 0001:0002372c       __ReadFont                 0003472c f libf:fontlib.obj
 0001:000238f8       __LoadFont                 000348f8 f libf:fontlib.obj
 0001:00023b20       __UnLoadFont               00034b20 f libf:fontlib.obj
 0001:00023b70       __unpload                  00034b70 f libf:fontlib.obj
 0001:00023bb4       __RegisterFont             00034bb4 f libf:fontlib.obj
 0001:00024354       __DrawChar                 00035354 f libf:fontlib.obj
 0001:00019e70       _OnTNT                     0002ae70 f libf:fhack.obj
 0001:00032a40       __get_fname                00043a40 f libc:fpexcept.obj
 0001:00031ea0       _flsall                    00042ea0 f libc:FFLUSH.OBJ
 0001:00030c30       __before                   00041c30 f libc:HEAPADD.OBJ
 0001:000307d0       __abstract_cw              000417d0 f libc:ieee87.obj
 0001:00030880       __hw_cw                    00041880 f libc:ieee87.obj
 0001:00030930       __abstract_sw              00041930 f libc:ieee87.obj
 0001:0002efd0       _comexecmd                 0003ffd0 f libc:SPAWNVE.OBJ
 0001:0002db50       __heap_new_region          0003eb50 f libc:HEAPGROW.OBJ
 0001:0002d810       __cftoe_g                  0003e810 f libc:cvt.obj
 0001:0002d940       __cftof_g                  0003e940 f libc:cvt.obj
 0001:0002daa0       __shift                    0003eaa0 f libc:cvt.obj
 0001:0002d240       _parse_cmdline             0003e240 f libc:STDARGV.OBJ
 0001:0002d090       _xcptlookup                0003e090 f libc:WINXFLTR.OBJ
 0001:0002c670       _ctrlevent_capture@4       0003d670 f libc:WINSIG.OBJ
 0001:0002c970       _siglookup                 0003d970 f libc:WINSIG.OBJ
 0001:0002c450       _findenv                   0003d450 f libc:PUTENV.OBJ
 0001:0002af20       __make_time_t              0003bf20 f libc:MKTIME.OBJ
 0001:0002ab20       __timet_from_ft            0003bb20 f libc:FINDFILE.OBJ
 0001:0002a650       __getextendedkeycode       0003b650 f libc:GETCH.OBJ
 0001:00029a60       _xtoa                      0003aa60 f libc:XTOA.OBJ
 0001:000296d0       _doexit                    0003a6d0 f libc:CRT0DAT.OBJ
 0001:00029750       __initterm                 0003a750 f libc:CRT0DAT.OBJ
 0001:000291f0       __heap_expand_block        0003a1f0 f libc:REALLOC.OBJ

FIXUPS: 29e58 29 a 4b0 fffffc8a 15 2d 20 d 23 c f 23 f 52 73 13 14 f 2a
FIXUPS: 2a1d8 fffffd92 ffffff77 5 fffffec1 a a 34 5 5 5 5 1e 9 19 b82 ffffff61
FIXUPS: 2a930 6 ffffffdc fffffff7 ffffffef ffffffde ffffffe6 fffffff7 fffffff4
FIXUPS: 2a8a1 ffffffd5 ffffff1f 5f fffffe62 12 12 20 1d 10 5e 12 11 fffffdb6
FIXUPS: 2a51f fffffe6c fffffee7 f e c 3f cb2 fffffff6 fffffff6 fffffff6
FIXUPS: 2af64 ffffffe8 fffffff6 ffffffe8 ffffffe8 fffffff6 ffffffe8 fffffff6
FIXUPS: 2aece ffffffe8 ffffffe8 ffffffe8 ffffff53 1b 3c 37 fffffd14 27
FIXUPS: 2abb7 17 1a b6 3f fffffe0f 15 33 1f fffffe42 e49 17 80 ffffff0a
FIXUPS: 2b45c d 1d 2a 31 11 d 5a 18 25 37 1a 12 fffffd97 fffffcca 26 17
FIXUPS: 2b164 9 19 15 31 2e 47 fffffd97 9 11 a ee1 fffffec9 e a 18 ffffff95
FIXUPS: 2bd79 a fffffe2a 1c b 1e 18 6e 1e 67 2e 9 fffffb74 c 9f 10 10 64
FIXUPS: 2b9e0 a3 10 10 53 4c 48 fffffc47 14ac fffff90c 9e 30 47 47 182
FIXUPS: 2c883 fffffbc3 18 61 fffffea8 1e 12 4f 20 13 fffffd7e 24 18 1d
FIXUPS: 2c20a fffffcfe 10 1f0 13 28 13 fffffc96 16 5c 1e 1182 79 28 2e
FIXUPS: 2cdd8 8d 3c 20 4a fffffdec c d 9 9 c d fffffb77 24d 4e c 6 16 a
FIXUPS: 2cb84 6 2b 3b 20 22 15 e 1a a99 46 34 b4 4b fffffc5d 40 79 28 2e
FIXUPS: 2d2a7 1c 35 33 3d 33 39 42 6 50 fffffcaa 39 1a 33 1f 2d 10 9 9
FIXUPS: 2d223 12 fffffd89 1177 11 fffffe22 11e fffffec6 fffffff1 ffffffd6
FIXUPS: 2defb fffffff6 ffffffc0 ffffffe2 ffffffd7 ffffffc5 fffffff3 fffffff7
FIXUPS: 2de10 ffffffe9 fffffff2 ffffffe2 ffffff70 13 2d 17 fffffeec 4d
FIXUPS: 2dd16 fffffdae 9 36 ab 9 51 b46 de 60 28 1f 17 31 3c 2a 3a 4c 15
FIXUPS: 2ea53 1d 1d 35 fffffad9 ffffff3d 11 32 25 b fffffe70 8d 14 fffffd4b
FIXUPS: 2e1d5 14 10 1c fffffedd 16 16c3 12 2e 12 fffff984 fffffe5d 1d 72
FIXUPS: 2f0ab 34 d 12 d fffffa1d e 52 2b d 8f e e d c 3a 9 fffffe0c fffffae8
FIXUPS: 2e5e0 d2 f 46 15 1b23 13 fffff7e7 e8 a8 138 55 da 63 10c 14 fffff328
FIXUPS: 2f2f3 70 12 1a9 1c 21 15 1e 24 e 11 14 18 19 2f 6b 20 4f 6c 12
FIXUPS: 30568 ffffffb6 fffffffb fffffff1 fffffff0 fffffff3 ffffff0c ffffffea
FIXUPS: 303db ffffffd9 fffffffb fffffff1 fffffff2 ffffffe5 fffffff4 ffffffd4
FIXUPS: 30333 ffffffe4 fffffcd7 27 f d 22 11 1f 25 81 13 25 24 83 2a 6a9
FIXUPS: 308bc ffffffa2 fffffff7 fffffffa ffffffea ffffff4e ffffffd1 fffffff9
FIXUPS: 3071a fffffffb ffffffab fffffffb ffffffe8 fffffffb ffffffdd ffffffbf
FIXUPS: 30635 ffffffea fffffff0 fffffff3 fffffff4 fffffffb fffffffb fffffff1
FIXUPS: 305d0 fffffff3 fffffff7 ffffffef fffffff9 fffffff5 ffffffda cda
FIXUPS: 3125a d 10 6 fffffdb0 29 56 11 1f 75 fffffe78 3b fffffdb2 ffffff78
FIXUPS: 30d22 fffffff8 fffffe51 13 13 74 88 9 6 27 2b fffffd2c fffffff6
FIXUPS: 3090f ffffffe3 fffffffb fffffff5 1199 76 43 29 d 43 3b a2 fffffce9
FIXUPS: 3170f 21 20 19 27 fffffe93 26 38 fffffe4a d 2c 2b 1f fffffe2d 58
FIXUPS: 31424 2c fffffee5 1d fffffe52 17 4c 32 1723 fffffbd6 160 34 1d
FIXUPS: 3233e cb 7 c d 1f 15 f a 15 1f fffffba4 4f 47 175 fffffaa9 15 1a
FIXUPS: 31d4b fb 9 e 9 25 47 fffffb56 29 1e15 bb 1c 2d 52 d d 1b d fffff60f
FIXUPS: 32f41 fffffe9b b 1d 4b 44 34 19 31 e fffffe56 1e 19 10 ffffff04
FIXUPS: 32b3a d4 2b fffffc85 65 12 18 1584 c 1c ffffff7a ffffffb8 9 e fffffdd4
FIXUPS: 33d89 1a fffff2d3 1f 5e 22 30 2e 13 44 f 12 30 4c f 4f f 15 14e
FIXUPS: 3358f f 114 21 29 fffe27e5 5d 6 11 c 24 14 6d 3b 61 c 43 28 41
FIXUPS: 16170 ab 1b 1f 30 30 30 30 30 ef 77 f0 32 7d 83 7a 1d7de ffffffa1
FIXUPS: 16b2c 20 e 63 14 7e 19 2b 1f 71 1e 16 12 7b 4d fffff98c 15c 121
FIXUPS: 15b1b 123 12 70 57 c 58 13 2b 11 2b 14 48 5a 187c 4b 12 34 fffffec8
FIXUPS: 1756f 2b 19 12 24 fffffa94 57 5 25 c 2c d bc 87 14c 95 22 fffff9fc
FIXUPS: 16ed8 19 c 1b 3c 4a b fffffb33 30 15cd 6 13 1d 13 7a 1a fffff9e4
FIXUPS: 17bd2 73 25 14 18 53 2b c8 2f fffffd0f ffffff4c 2b ffffff03 14
FIXUPS: 17901 13 12 10 a fffffea3 16 28 fffffecd 30 fe9 1a fffffc7a 14
FIXUPS: 183d2 15 1d d 3c 23 13 1b 1d 9 d 1d f 9 d 31 1a f fffffca5 aa 1f
FIXUPS: 18331 fffffb37 4f fd 38 25 bc cde fffffff4 fffffff0 ffffffeb ffffffee
FIXUPS: 18d56 fffffff8 fffffff0 ffffffd9 ffffffdc fffffff4 fffffff0 ffffffd9
FIXUPS: 18c8a fffffff4 ffffffef ffffffdf ffffffc4 ffffffea ffffffe0 ffffffec
FIXUPS: 18baa ffffffe3 ffffffe7 fffffa36 30 16 19 d 48 4e 1b 357 ffffffea
FIXUPS: 189b5 ffffffc2 ffffffd8 fffffff0 ffffffdc ffffffea ffffffe6 ffffffec
FIXUPS: 188bf fffffff8 ffffffea ffffffe6 ffffffe6 ffffffe6 ffffffe6 ffffffe6
FIXUPS: 18805 ffffffe6 ffffffe6 ffffffe3 ffffffe6 ffffffe6 ffffffe6 ffffffe6
FIXUPS: 18e91 ffffffc8 ffffffdb ffffffc5 ffffffea ffffffe1 6bc 1f 23 25
FIXUPS: 19543 1c 24 30 35 fffffd31 fffffe46 ffffff59 ffffffae fffffff5
FIXUPS: 19056 fffffffb ffffffe6 ffffffe9 fffffff5 fffffffb fffffff9 fffffff5
FIXUPS: 18ff9 fffffffb ffffffe4 fffffff3 ffffffea ffffff71 ffffffd2 fffffc22
FIXUPS: 18b04 ffffffe2 161b 29 18 d 10 29 5 1a 46 fffff8bd 89 10 3c fffffd4b
FIXUPS: 1994d 104 14 d 10 fffffd39 6f 29 fffffdf9 86 2b 3a 1b 20 c fffffc38
FIXUPS: 1944a 11 1151 22 1b 69 96 5d fffff4eb a1 1a d 3b 10 32 2c 5 83
FIXUPS: 19e6b a 1c 30 1c 37 33 16 39 12 7f 1a 10 2f 11 16 1269 fffff801
FIXUPS: 1ac2f 20 20 20 20 20 36 74 19 22 12 23 1c 3b fffffac4 39 77 43
FIXUPS: 1aa7b 15 fffffd7b 71 45 ffffff12 fffffbd6 90 37 2d 31 af 10ce 25
FIXUPS: 1ae7a 4b 12 18 29 d 10 2e 12 18 40 12 18 4c 12 18 40 1f 36 16 18
FIXUPS: 1b199 2b d 25 24 24 16 16 16 894 1d 13 12 38 1a 25 24 d d 4e 81
FIXUPS: 1bd17 fffff970 19 c f 27 fffffd88 4f 43 c 6 18 23 42 25 1c c 6
FIXUPS: 1b5f6 23 86c fffffff4 ffffff7d ffffffdc fffffff1 fffff964 12 30
FIXUPS: 1b796 1e 21 15 19 f f b6 2e 3a f 57 1b 1a 2a 14 25 1e f d 3a 1c
FIXUPS: 1bae1 1c bb5 1c 8 c 19 2f 26 c 1e 34 c 20 28 c 20 38 c fffffa71
FIXUPS: 1c2d3 ffffffb3 fffffec5 ffffff80 ffffff8b fffffff0 ffffffd1 ffffff6e
FIXUPS: 1bf70 fffffff4 ffffffef ffffff92 ffffffe2 ffffffcd a82 39f fffffbf2
FIXUPS: 1c8a2 fffffff5 fffffa98 11 36 16 1d 8 9 18 11 2e 4f 1d 34 34 3a
FIXUPS: 1c54f 2a 34 25 18 c 20 18 c 1f 48 8 e40 c2 5e 19 fffff9d4 ffffff52
FIXUPS: 1cf32 ffffffe8 ffffffe5 fffffff5 fffffff3 ffffffc0 fffffff2 fffffff9
FIXUPS: 1ce6b fffffffb fffffffb ffffffb1 ffffffe7 ffffffc6 fffffff9 fffffffa
FIXUPS: 1cd79 ffffffbb ffffffc5 ffffff5a ffffff0d ffffffda ffffff25 ffffff52
FIXUPS: 1c9aa ffffffca 242f 47 1d 12 1c 10 13 73 2f 6 88 2a 24 e ffffe17f
FIXUPS: 1d16b 1a 2e f 22 39 1f 11 12 8 12 3e 7b 135 8 e a 1387 6f 12 c
FIXUPS: 1e8b1 67 38 4b 24 7b 29 3c 1c 6 13 20 1d 42 46 c 9 23 d d d d d
FIXUPS: 1eca7 26 2e 4c 3c fffff3ba c 6c 1a b3 18 16 24 66 2d 41 3e a 16
FIXUPS: 1e41f 6 18 90 c2 9 15 16 18 53 33 32 52 2c 15 3a 68 2a fffff448
FIXUPS: 1dc51 18 17 19 17 19 3d 5 51 19 66 42 17 32 f a 14 1d 14 11 a f
FIXUPS: 1defa e2 19 24 18 12 3d 45 4a fffff5de 30 3d 10 41 53 12 66 11
FIXUPS: 1d893 23 a 3f 2a 10 1f a 10 e 11 3f 13 23 a 3f 2a 10 1f a 10 e
FIXUPS: 1dae1 2411 d fffff8cf 32 37 ce b 16 fe 6 d 1e 7f 16 fffffb1f 1e
FIXUPS: 1f734 fffffcb8 b 25 3d 24 75 14 fffffe3a fffffe6c 23 79 b 3c 2f
FIXUPS: 1f2cc 1236 52 8 20 19 32 26 21 23 34 1c 16 fffffdb4 c 17 fffffd09
FIXUPS: 20209 83 fffffdbc fffffbc6 229 2c d d d d d d d d d d f02 54 1d
FIXUPS: 2118f d 126 34f 13 1c 16 fffff611 fffffe2e 147 e e fffffb3b 15
FIXUPS: 2080c 9 e 9 29 1b d 40 28 31 17 2b 40 1f fffffb38 2091 fffffff9
FIXUPS: 2252d ffffff38 fffffff9 ffffffd9 fffffff9 ffffffde fffffff9 ffffffae
FIXUPS: 223ae ffffffb6 fffffff9 ffffff91 fffffff9 ffffffbe fffffff9 fffffb8f
FIXUPS: 21dd6 fffffbe3 fffffeb1 fffffed1 ffffffe6 ffffff90 5ec ffffffef
FIXUPS: 21c87 fffffff9 ffffff48 fffffffb fffff15d 3c 287d 15 18 fffffeb8
FIXUPS: 23499 ffffffda fffff58d ffffff61 ffffffc3 ffffff2e 45b fffffff9
FIXUPS: 22ca1 fffffff2 ffffff28 ffffff29 745 fffffee6 fffffe84 ffffffbd
FIXUPS: 22f12 485 fffffffb ffffffc0 fffffffb ffffff6a ffffeeec ffffffea
FIXUPS: 22171 ffffffc7 ffffffde ffffff57 1fba ffffffdc fffffff5 fffffff4
FIXUPS: 23fb1 fffffff5 ffffffed ffffff90 fffffff5 ffffffea ffffffee ffffffe3
FIXUPS: 23eb8 ffffffe6 fffffffb fffffff4 ffffffc9 fffffb40 fffffffb fffffd18
FIXUPS: 236b2 2f 20 2f 15 19 fffffee7 14 18 ffffff02 24 1f 1110 ffffffe8
FIXUPS: 24689 fffffff0 ffffffe7 ffffffee fffffff0 ffffffec fffffff0 ffffff34
FIXUPS: 244a7 fffffff9 ffffffe1 ffffffdd ffffffef ffffffea ffffffdc ffffffeb
FIXUPS: 243ef ffffffd0 fffffff4 ffffffdd fffffff6 ffffff9f ffffffb4 ffffffdc
FIXUPS: 24252 ffffff5f ffffffe3 ffffffe8 ffffff69 ffffff53 e45 f a 3f b
FIXUPS: 24f9a 10 9 18 a3 5f 13 27 dd 44 13d 195 2d 5b 53 58 a 18 42 2e
FIXUPS: 256ca f 17 4d 40 7f ffffeeda 213 3e 65 48 20 1e 6d 1f 38 27 13
FIXUPS: 24b31 27 35 b f 3e 25 f 21 f 12 f 13 f 1c 2c 27 4e 5d 75 4b 1504
FIXUPS: 26388 19 1b 16 61 2a 19 1a 19 fb 8 20 1b 6c f 18 6e 8 18 b b b
FIXUPS: 26734 1b fffff295 ffffed5a 49 13 19 107 16 13c0 4f 52 d3 136 2a
FIXUPS: 25f8f 29 2a 20 b b b 11 21 40 2d 17 20 17 2b 25 28 3d 2b 96 27
FIXUPS: 262d4 19 33 16 1b eda ffffffde ffffffb7 fffff667 10 d a e 10 10
FIXUPS: 2688c 10 10 10 10 ffffff47 ffffffed ffffffed ffffffee ffffffed
FIXUPS: 267b4 ffffffed ffffffed ffffffee ffffffed fffff38c 94 4a c 2b 8
FIXUPS: 25c64 1d29 fffffff1 ffffffef ffffffe4 ffffffba ffffffaf fffffe47
FIXUPS: 27573 ffffff29 ffffffe0 ffffffa7 fffffff8 fffffd2f fffffff8 fffffffb
FIXUPS: 27137 ffffffeb fffffff9 ffffffe2 ffffffc6 ffffff5e ffffff3b ffffff41
FIXUPS: 26e38 ffffffbc 586 ffffffce ffffffd7 ffffff32 fffffff9 fffffffb
FIXUPS: 27232 13d2 63b ffffff01 ffffff0e ffffffe2 ffffffd1 ffffffac ffffffaa
FIXUPS: 2909f fffffff0 ffffffbe ffffffaf ffffff92 ffffff4f ffffffde ffffff6f
FIXUPS: 28e23 ffffffb1 ffffffde ffffff76 fffffff9 49f ffffffef ffffffbf
FIXUPS: 290df fffffff9 ffffecb3 1d 26 14 fffffd78 ffffffc9 201f ffffff04
FIXUPS: 29a31 ffffffe3 ffffffda ffffffd6 ffffffe3 ffffff9a fffffc73 ffffffeb
FIXUPS: 29594 ffffff23 fffffde4 fffffffb ffffffe0 fffffffb fffffffb fffffff9
FIXUPS: 29247 ffffffa0 fffff6bc ffffffec fffffff9 ffffffcb ffffffc1 ffffffef
FIXUPS: 287fc ffffffa4 fffffff9 ffffff7d fffffff9 ffffff19 fffdc329 10
FIXUPS: 4983 d 52 3d 8 7c 43 24 12 16 5a 43 81 1f 23 26 1c d 1c 3e 13 e
FIXUPS: 4d68 1e 3e 13 e c 24 ffffc1f7 2e8a 1c 1b9 19 138 12 98 11a b f2
FIXUPS: 44ea 10 57 3d 8 7c 17 4f 29 3e 13 e 1e 3e 13 e c 68 12 16 1e ad
FIXUPS: 2d92 1c 12d 6dd d 12 d6 123 150 23 12 36 33 13 31 1c 1c 53 2f d1
FIXUPS: 3be3 2f d1 28 29 22 56 22 56 27 12 27 ffffe814 23 d 9d d 2d 39
FIXUPS: 2835 d d6 39 81 95 27 1b 33 32 12 16 23 32 4d 38 a 2d 2a f 12 14
FIXUPS: 2cc7 41 56 ffffecc9 14 1a 15 d c 1d 27 52 2e 121 e 67 4d 29 26
FIXUPS: 1e17 74 d 57 20b d d 1c 69 313 db f 31 f 1e 17 ffffef63 21 12 24
FIXUPS: 15e9 1c 38 13 e 1e 23 c 21 21 54 1f 3c 17 13 1e 1e 1e 23 54 41
FIXUPS: 192f d 6b 2e 17 15 14 579d 13d c0 13d 6d 50 79 fb 12c 7a 52 24
FIXUPS: 79a3 1c 93 2a9 12a 73 17d fc 20 60 7f ffff9299 f 1a c 1f 11 1b
FIXUPS: 1544 1b 4aca 93 322 b1 6b fc 10 60 44 c7 13f 14d 62 42 3a 32 47
FIXUPS: 6b63 38 15 1b 20 16 bf 10d 4c 20 2f be 1e 82 3c ffffdf1e 2c bb
FIXUPS: 5018 64 d 23c 50 fc 116 512 3a d 37 d 37 1d c4 3e 3e 31 5c 4c 17
FIXUPS: 5d72 3d 124 f 12 1f 44 2a 384c 94 2b cc 2e 6f 235 33 188 ec 20
FIXUPS: 9f10 1c 8c d2 94 2b 1a 12 12 124 2e 33 32 5a 11 19 d ffffaa6a 98
FIXUPS: 4ee2 27 33c4 4a 28 19 93 42 192 d 1d 4a 196 16 19 179 28 2d 1a
FIXUPS: 89f6 20 28 151 165 24 aa af 3f 383 cb 5a 49 1ec 175 1c1b da 58
FIXUPS: b46a 67 11a 18 6c a2 e 6c 17 16 1c 71 d 6d 42 12 4f 6c b0 10f 27
FIXUPS: bbce 5f 12 16 ffffc5d4 11 43 1c 4f26 fd ffffd13d e7 32 e5 5e 75
FIXUPS: a9a4 76 85 1d7 1c b1 20 cd 67 d2 66 60 8d 48 19 54 12 d 1c 71 d
FIXUPS: b255 d 4f fbf 11 b4 11 15 19 54 16 51 82 14 20 c0 35 b0 c5 15 1d6
FIXUPS: c986 38 fa 1e 4c 12 94 5d 65 6b 19 2b8 1e 64 51e 25 20 17 21 67
FIXUPS: d694 22 6a 62 1b 142 59 ae 7b 5a 12 fffff80c ffffe9a0 7d 1e 16
FIXUPS: bd5a d 99 51 96 12 12d 1c 123 9e 78ed 22 21 13 18 ffffa4db 21 1a
FIXUPS: e085 14 35 3d fffffe3c 3c 3f 5d fffffaca 12d 31 48 4e 2e 48 4e
FIXUPS: ddcf 39 39 5c 17 4e 17 fffff5f0 32f0 37e 1a6 e 2b8 179 1e6 1c 2b2
FIXUPS: 1162e 41c 4f 2e 71 37 1c 126 4e 18b 535 2cd c8 3fe 268 263 51c
FIXUPS: 13a2c 8 55 c 1e 16 ffffb3a6 26 23 12c 23 a0 a1 224 1af 1c a1 224
FIXUPS: f9ab 1c a1 28a 52 ec 1fb 15a 58 11 69 b 15 2b 1a6 89 e 239 b cb
FIXUPS: e585 c 1e 16 3c c 81 1c 4f 11 2d 35 ab 4e a8 5e 12 35 1c a5 d 26
FIXUPS: eb04 88 1a 1e 12c 1c 3e 5d 85 1b 4e92 f 217 fffffc9a 43 75 ffffa4fa
FIXUPS: e234 36 8 59 c 1e 16 27 23 13 18 23 1c 8 56 c 1e 16 27 22 21 13
FIXUPS: e4f2 31 c 6b0f 11 fffffdda bd fffffe63 ba fffffd46 af 1d 10e fffff9d6
FIXUPS: 14708 88 8b e0 167 b5 11 fffffb84 20 fffffd8d 54 1ca 11 fffffb81
FIXUPS: 14259 1c6 11 fffffb19 124 c3 be 167b a3 32 cc fffffddf f 15 31
FIXUPS: 1584e ffffff60 fffffeab cf 1c 22 fffffc53 f 35 1a 15 d fffffea0
FIXUPS: 1533e fffffebb 64 fffffe1c 5c 64 88 16 fffffd32 82 2a
